S0220000687474703A2F2F737265636F72642E736F75726365666F7267652E6E65742F1D
S12300000C9465000C940D250C9403250C9482000C9482000C9482000C9482000C94820093
S12300200C9482000C9482000C9482000C94A2240C9482000C94CF240C94F9240C94EF24CB
S12300400C9467240C9482000C941A240C9482000C94C4250C948C250C9482000C94820031
S12300600C9482000C9482000C9482000C94820008000000BE922449123EABAAAA2ABECD2B
S1230080CCCC4C3E00000080BEABAAAAAA3E00000000BF000000803F0000000000084178D6
S12300A0D3BB4387D1133D190E3CC3BD4282AD2B3E68EC8276BED98FE1A93E4C80EFFFBE54
S12300C001C4FF7F3F000000000011241FBECFEFD0E1DEBFCDBF12E0A0E0B1E0E8E4FFE73B
S12300E002C005900D92A831B107D9F716E0A8E1B2E001C01D92AE31B107E1F70E94A20E63
S12301000C94A23F0C940000282F392FEFE3F0E0808181FDFDCF822F932F92BD81BDF89A7C
S123012080B50895282F392FEFE3F0E0808181FDFDCF1FBA822F932F92BD81BD60BD0FB682
S1230140F894FA9AF99A0FBE0895EAE7F0E0108210927C0080E880BF85EE808311B812B87D
S1230160A5E5B2E020E030E04AEF53E42D933D934D935C931397E1E3F2E084EF91E0918348
S123018080833A969183808354962D933D934D935C9313970895CF92DF92EF92FF920F935B
S12301A01F93CF93DF93282FEA01F89480919502882349F0213039F480918F02893019F079
S12301C041155105B9F580E090E0C22EDD24E090A901F090AA010091AB011091AC0124E626
S12301E030E040E050E00E94F73E6E0D7F1D801F911FCC0CDD1CCC0CDD1CF601E655FD4F3E
S12302006083718382839383BE0180E090E0E080F180028113810E94F73E6E0D7F1D801FE4
S1230220911F22ED32E0C20ED31EF60160837183828393837894DF91CF911F910F91FF9084
S1230240EF90DF90CF9008950F931F93CF93DF93082F10E0F801EE0FFF1FE55DFD4F8081BE
S12302609181835F93400CF05EC0F801EE0FFF1FE55DFD4F808191818F5D934014F088EDAC
S123028053C040E050E0C801880F991FDC01A55DBD4F6BE571E02D913C911197EA01CA016A
S12302A0880F991FFB01E80FF91F808191818217930798F5CA010197ABE5B1E0880F991F3A
S12302C08A0F9B1FFC0120813181F801EE0FFF1FE55DFD4F00811181FC0160817181CA0127
S12302E0880F991FA80FB91F4D915C91201B310BC901880F991F880F991F641B750B820FE2
S1230300931F0E94223FCE01880F991F880F991F8C0F9D1F8D97860F07C04F5F5F4F47320B
S1230320510509F0B8CF86E9DF91CF911F910F9108958091F2029091F302A091F402B09134
S1230340F5020097A105B10509F057C080918F028E3161F18F3140F48A30C1F08431F1F0F7
S1230360893009F04AC00AC0803281F1803230F18832A1F1833609F040C038C088E06AE054
S123038070E04AE050E00E94CB0037C088E065E070E045E050E00E94CB002FC088E060E0F5
S12303A070E042E350E00E94CB0027C088E06EE170E04AE050E00E94CB001FC088E064E1E6
S12303C070E04AE050E00E94CB0017C088E064E170E04AE050E00E94CB000FC088E062E3EB
S12303E070E04AE050E00E94CB0007C088E064E670E04AE050E00E94CB00809133029091EB
S123040034028D549440ACF08091F6029091F702A091F802B091F9020097A105B10509F0DB
S123042071C089E06AE070E04AE550E00E94CB00089580913D0290913E0289379105ACF078
S12304408091F6029091F702A091F802B091F9020097A105B10509F055C089E06AE070E00A
S123046046E450E00E94CB00089580919F029091A002892BA1F48091F6029091F702A09102
S1230480F802B091F9020097A105B10541F089E060E070E040E050E00E94CB00089580919A
S12304A09F029091A0020197A1F48091F6029091F702A091F802B091F9020097A105B1052A
S12304C041F489E064E170E04AE050E00E94CB00089580919F029091A002029799F48091D5
S12304E0F6029091F702A091F802B091F9020097A105B10539F489E06AE070E04AE050E002
S12305000E94CB000895EF92FF920F931F9388E10FB6F89480936000109260000FBE0E94C9
S1230520493680E091E00E9429360F2EFFEFEF2EFFE1FF2EFCE10F2FF0E01F2FF02DD801E2
S1230540C7010197A109B109000001F0D1F7C895000060912B0270912C026353714088275A
S123056077FD8095982F0E94683D9B01AC0163E373E387EA91E40E94CD3C60934F01709324
S12305805001809351019093520160914F0170915001809151019091520120E030E849E977
S12305A053E40E94613E609353017093540180935501909356018FE491E06CE271E00E9418
S12305C00A2783E591E060E371E00E940A272DE088E190E00FB6F894A895809360000FBEF2
S12305E020936000D801C7010197A109B109000001F0D1F7C89500001F910F91FF90EF90D3
S123060008954F925F926F927F928F929F92AF92BF92CF92DF92EF92FF920F931F937C01BC
S123062070E06B01CC0CDD1CC60ED71ECC0CDD1C86E295E0C80ED91EF601619171918080FA
S1230640918080E090E00E94663D2B013C0100E010E0C801B7010E94663D20E030E44CE928
S123066050E40E94613E9B01AC0160E070E48CE995E40E94CD3C20E030E040E85FE30E946F
S1230680643C9B01AC01C301B2010E94CD3C7B018C01AA24BB24C501B4010E94663D9B0139
S12306A0AC01C801B7010E94CD3C0E94213E7B018C01E4E0F0E0CE0EDF1EF601608171811C
S12306C080E090E00E94663D9B01AC01C801B7010E94CD3C22E63BEE4BE55BE30E94653CAA
S12306E09B01AC0160E070E080E89FE30E94CD3C20E030E848E853E40E94643C7B018C01BE
S123070020E030E046E153E40E94183E1816ACF0C801B70120E030E040E050E40E94C93C19
S123072088235CF0C801B70120E030E040E251E40E94613E0E94353D02C06CED75E0862F5C
S1230740972F1F910F91FF90EF90DF90CF90BF90AF909F908F907F906F905F904F9008954E
S1230760FF920F931F93CF93DF930E945A26F82E109290028823F1F0809190028F15A0F4D9
S1230780C0E4D5E00091900210E00E94F625FE01E00FF11F8083809190028F5F80939002F5
S12307A0809190028F1570F36091900280E495E00E94353410929002DF91CF911F910F91D0
S12307C0FF9008952F923F924F925F926F927F928F929F92BF92CF92DF92EF92FF920F934A
S12307E01F93CF93DF93F8948091A9019091AA01A091AB01B091AC018093FA029093FB0262
S1230800A093FC02B093FD0278940F2EF1EBEF2EF1E0FF2EF02DCC24DD2400E010E00F2E06
S1230820FAEA6F2EF2E07F2EF02D0F2EF5EC4F2EF1E05F2EF02D0F2EF2ED8F2EF2E09F2E09
S1230840F02D22243324B02EE801C801880F991F880F991FF301E80FF91F80819181A28173
S1230860B3810097A105B10509F47DC0CE01880F991F880F991FF301E80FF91F2081318150
S1230880428153818091FA029091FB02A091FC02B091FD02281739074A075B0708F063C0D6
S12308A0F701A081B1819C91F201EC0FFD1F8081892B8C93CE01880F991F880F991FF3017D
S12308C0E80FF91F1082118212821382F7E0F01708F449C08CE80E941A2685E00E941A2637
S12308E0802F0E941A2680918F0280680E941A266091FA027091FB028091FC029091FD02DD
S123090024E630E040E050E00E94493F822F0E941A266091FA027091FB028091FC02909191
S1230920FD0224E630E040E050E00E94493FBB27A52F942F832F0E941A266091FA02709125
S1230940FB028091FC029091FD0224E630E040E050E00E94493FCA01AA27BB270E941A2673
S123096083E70E941A26CE01880F991F880F991FF401E80FF91F80819181A281B3810097B5
S1230980A105B10509F47EC0CE01880F991F880F991FF401E80FF91F208131814281538161
S12309A08091FA029091FB02A091FC02B091FD02281739074A075B0708F064C0F701A08132
S12309C0B1819C91F201EC0FFD1F8081809589238C93F7E0FB1508F449C08CE80E941A2687
S12309E085E00E941A268B2D0E941A2680918F028F770E941A266091FA027091FB0280918C
S1230A00FC029091FD0224E630E040E050E00E94493F822F0E941A266091FA027091FB02A2
S1230A208091FC029091FD0224E630E040E050E00E94493FBB27A52F942F832F0E941A26E2
S1230A406091FA027091FB028091FC029091FD0224E630E040E050E00E94493FCA01AA2748
S1230A60BB270E941A2683E70E941A26CE01880F991F880F991FF401E80FF91F10821182CC
S1230A8012821382D701ED91FC919081F201EC0FFD1F80819101892311F021E030E0C90110
S1230AA002C0880F991FCA95E2F7C82AD92A0F5F1F4FE2E0F0E0EE0EFF1E0A30110509F024
S1230AC0C2CED0921F05C0921E05DF91CF911F910F91FF90EF90DF90CF90BF909F908F90EE
S1230AE07F906F905F904F903F902F9008951F9380914701813009F0A7C080911E0290917D
S1230B001F02A0912002B09121020097A105B105A9F48091A9019091AA01A091AB01B091C4
S1230B20AC0180509342A249BF4F80931E0290931F02A0932002B093210286C020911E021D
S1230B4030911F0240912002509121028091A9019091AA01A091AB01B091AC0128173907E7
S1230B604A075B0708F070C010918F028CE380938F02809133029091340290939B028093E1
S1230B809A028CE80E941A2685E00E941A2688E00E941A2680918F0280680E941A26609171
S1230BA0A9017091AA018091AB019091AC0124E630E040E050E00E94493F822F0E941A2629
S1230BC06091A9017091AA018091AB019091AC0124E630E040E050E00E94493FBB27A52FF5
S1230BE0942F832F0E941A266091A9017091AA018091AB019091AC0124E630E040E050E05E
S1230C000E94493FCA01AA27BB270E941A2683E70E941A2610938F028091A9019091AA013F
S1230C20A091AB01B091AC0180589141A94CBF4F80931E0290931F02A0932002B093210206
S1230C408091480180931D021F910895EF92FF920F931F93CF93DF93F894E090A901F09057
S1230C60AA010091AB011091AC01789440E050E0CAEAD2E062ED72E09A01CA01880F991F22
S1230C80880F991FFE01E80FF91F80819181A281B3810097A105B10531F1CA01880F991F5A
S1230CA0880F991FFE01E80FF91F80819181A281B381E816F9060A071B07A8F4CA01880F3B
S1230CC0991F880F991FFE01E80FF91F80819181A281B3818E199F09A00BB10B80839183C4
S1230CE0A283B3830CC0C901880F991F880F991FFE01E80FF91F1082118212821382C9013B
S1230D00880F991F880F991FFB01E80FF91F80819181A281B3810097A105B10531F1C901DD
S1230D20880F991F880F991FFB01E80FF91F80819181A281B381E816F9060A071B07A8F4D0
S1230D40C901880F991F880F991FFB01E80FF91F80819181A281B3818E199F09A00BB10BFC
S1230D6080839183A283B3830CC0C901880F991F880F991FFB01E80FF91F10821182128205
S1230D8013824F5F5F4F4A30510509F075CF2AEB32E0D9011D921D921D921D9282EE92E0B2
S1230DA0FC0111921192119211921D921D921D921C9213971082118212821382F90138962B
S1230DC01082118212821382FC0138961082118212821382F9013C9610821182128213828E
S1230DE0FC013C961082118212821382F90170961082118212821382FC017096108211825C
S1230E00128213822C5E3F4FF90110821182128213824496FC01108211821282138280910F
S1230E201E0290911F02A0912002B09121028E199F09A00BB10B80931E0290931F02A09335
S1230E402002B09321021092A6021092A7021092A8021092A90284E690E0A0E0B0E08093DB
S1230E608B0290938C02A0938D02B0938E020E94EE3B8CE80E941A2685E00E941A2689E0CA
S1230E800E941A2680918F0280680E941A26C801B70124E630E040E050E00E94493FE22EDB
S1230EA0F32E042F152F822F0E941A26BB27A12F902F8F2D0E941A267801002711278E2D61
S1230EC00E941A2683E70E941A26F89484E190E0A0E0B0E08093A9019093AA01A093AB0105
S1230EE0B093AC018093AD019093AE01A093AF01B093B0017894DF91CF911F910F91FF90D9
S1230F00EF9008950F931F93CF93DF93E1E9F3E08CEB92E09183808380E293E090931204DE
S1230F20809311049F01265F3F4F80E090E0A7EDB3E4E90188839983AA83BB83CF010296F3
S1230F400E94DC2B80E090E0A0EAB0E480931B0390931C03A0931D03B0931E0303E113E0F5
S1230F60C8010E94DC2B0C5F1F4FF801108212BC11BCDF91CF911F910F9108950F931F93EB
S1230F80CF93DF9302E910E084E090E06CED70E0A8010E944F3C86E090E062E070E0A8013A
S1230FA00E944F3C88E090E063E770E0A8010E944F3C8AE090E062E270E0A8010E944F3C74
S1230FC08CE090E064E070E0A8010E944F3C8EE090E06EE170E0A8010E944F3C80E190E0A3
S1230FE060E773E0A8010E944F3C82E190E06EE170E0A8010E944F3C84E190E068E770E0C1
S1231000A8010E944F3C86E190E068EC70E0A8010E944F3CEFE3F0E0808181FDFDCF1FBADF
S123102088E190E092BD81BD88E280BD0FB6F894FA9AF99A0FBEEFE3F0E0808181FDFDCF6D
S12310401FBA89E190E092BD81BD81E480BD0FB6F894FA9AF99A0FBEEFE3F0E0808181FD44
S1231060FDCF1FBA8AE190E092BD81BD81E480BD0FB6F894FA9AF99A0FBEEFE3F0E08081D5
S123108081FDFDCF1FBA8BE190E092BD81BD85E080BD0FB6F894FA9AF99A0FBEEFE3F0E037
S12310A0808181FDFDCF1FBA8CE190E092BD81BD81E480BD0FB6F894FA9AF99A0FBEEFE3E5
S12310C0F0E0808181FDFDCF1FBA8DE190E092BD81BD86E480BD0FB6F894FA9AF99A0FBEC1
S12310E002E910E08EE190E064E170E0A8010E944F3C80E290E06EE170E0A8010E944F3C80
S123110082E290E068EC70E0A8010E944F3CEFE3F0E0808181FDFDCF1FBA84E290E092BD92
S123112081BD84E180BD0FB6F894FA9AF99A0FBEEFE3F0E0808181FDFDCF1FBA85E290E0E9
S123114092BD81BD84E180BD0FB6F894FA9AF99A0FBEEFE3F0E0808181FDFDCF1FBA86E2E9
S123116090E092BD81BD80E580BD0FB6F894FA9AF99A0FBEEFE3F0E0808181FDFDCF1FBAC1
S123118087E290E092BD81BD82E380BD0FB6F894FA9AF99A0FBEEFE3F0E0808181FDFDCF11
S12311A01FBA88E290E092BD81BD88E280BD0FB6F894FA9AF99A0FBEEFE3F0E0808181FDDE
S12311C0FDCF1FBA89E290E092BD81BD86E080BD0FB6F894FA9AF99A0FBEEFE3F0E0808173
S12311E081FDFDCF1FBA8AE290E092BD81BD10BC0FB6F894FA9AF99A0FBEEFE3F0E08081AB
S123120081FDFDCF1FBA8BE290E092BD81BD8AE080BD0FB6F894FA9AF99A0FBEEFE3F0E0AF
S1231220808181FDFDCF1FBA8CE290E092BD81BD82E180BD0FB6F894FA9AF99A0FBEEFE364
S1231240F0E0808181FDFDCF1FBA8DE290E092BD81BD8AE080BD0FB6F894FA9AF99A0FBE3E
S1231260EFE3F0E0808181FDFDCF1FBA8EE290E092BD81BD10BC0FB6F894FA9AF99A0FBE26
S1231280EFE3F0E0808181FDFDCF1FBA80E390E092BD81BD8DE280BD0FB6F894FA9AF99A00
S12312A00FBEEFE3F0E0808181FDFDCF1FBA81E390E092BD81BD83E080BD0FB6F894FA9AB1
S12312C0F99A0FBEEFE3F0E0808181FDFDCF1FBA82E390E092BD81BD81E080BD0FB6F89493
S12312E0FA9AF99A0FBEEFE3F0E0808181FDFDCF1FBA83E390E092BD81BD86E080BD0FB665
S1231300F894FA9AF99A0FBEEFE3F0E0808181FDFDCF1FBA84E390E092BD81BD86E080BD7C
S12313200FB6F894FA9AF99A0FBEEFE3F0E0808181FDFDCF1FBA85E390E092BD81BD81E0D8
S123134080BD0FB6F894FA9AF99A0FBEEFE3F0E0808181FDFDCF1FBA86E390E092BD81BDDB
S123136081E080BD0FB6F894FA9AF99A0FBEEFE3F0E0808181FDFDCF1FBA87E390E092BD97
S123138081BD10BC0FB6F894FA9AF99A0FBEC4E6D0E002E910E0CE0168EE73E0A8010E9402
S12313A04F3CCE01029668E97AE3A8010E944F3CCE0104966CE37FE0A8010E944F3C2C9604
S12313C0C439D10541F727E436E0EFE3F0E0C1E4D0E0A0E4B0E0808181FDFDCF1082C9012B
S12313E00397998388831C920FB6F894FA9AF99A0FBE808181FDFDCF1082C90102979983D9
S123140088831C920FB6F894FA9AF99A0FBE808181FDFDCF1082C9010197998388831C92B6
S12314200FB6F894FA9AF99A0FBE808181FDFDCF1082398328831C920FB6F894FA9AF99AF9
S12314400FBE2C5F3F4F86E02B35380709F0C3CFEFE3F0E0808181FDFDCF1FBA80E496E072
S123146092BD81BD10BC0FB6F894FA9AF99A0FBEEFE3F0E0808181FDFDCF1FBA81E496E029
S123148092BD81BD10BC0FB6F894FA9AF99A0FBEEFE3F0E0808181FDFDCF1FBA82E496E008
S12314A092BD81BD10BC0FB6F894FA9AF99A0FBEEFE3F0E0808181FDFDCF1FBA83E496E0E7
S12314C092BD81BD10BC0FB6F894FA9AF99A0FBEDF91CF911F910F910895CF92DF92EF925A
S12314E0FF920F931F93EFE3F0E0808181FDFDCF85E090E092BD81BDF89A80B58F3F11F41A
S12315000E94BE07EFE3F0E0808181FDFDCF84E090E092BD81BDF89A30B5EFE3F0E08081F8
S123152081FDFDCF85E090E092BD81BDF89A20B5922F80E0830F911D9093120180931101D8
S1231540EFE3F0E0808181FDFDCF86E090E092BD81BDF89A30B5EFE3F0E0808181FDFDCFD3
S123156087E090E092BD81BDF89A20B5922F80E0830F911D9C01220F331F880F991F880F35
S1231580991F880F991F280F391F3093340120933301EFE3F0E0808181FDFDCF88E090E00D
S12315A092BD81BDF89A30B5EFE3F0E0808181FDFDCF89E090E092BD81BDF89A20B5922FA8
S12315C080E0830F911D9C01220F331F880F991F880F991F880F991F280F391F30931401F3
S12315E020931301EFE3F0E0808181FDFDCF8AE090E092BD81BDF89A30B5EFE3F0E08081B2
S123160081FDFDCF8BE090E092BD81BDF89A20B5922F80E0830F911D9C01220F331F880F95
S1231620991F880F991F880F991F280F391F3093160120931501EFE3F0E0808181FDFDCF31
S12316408CE090E092BD81BDF89A30B5EFE3F0E0808181FDFDCF8DE090E092BD81BDF89ABD
S123166020B5922F80E0830F911D9C01220F331F880F991F880F991F880F991F280F391F94
S12316803093180120931701EFE3F0E0808181FDFDCF8EE090E092BD81BDF89A30B5EFE3FE
S12316A0F0E0808181FDFDCF8FE090E092BD81BDF89A20B5922F80E0830F911D9C01220F09
S12316C0331F880F991F880F991F880F991F280F391F30931C0120931B01EFE3F0E08081E6
S12316E081FDFDCF80E190E092BD81BDF89A30B5EFE3F0E0808181FDFDCF81E190E092BDB9
S123170081BDF89A20B5922F80E0830F911D9093580180935701EFE3F0E0808181FDFDCFEB
S123172082E190E092BD81BDF89A30B5EFE3F0E0808181FDFDCF83E190E092BD81BDF89AEE
S123174020B5922F80E0830F911D9C01220F331F880F991F880F991F880F991F280F391FB3
S123176030931E0120931D0184EB90E09093220180932101EFE3F0E0808181FDFDCF84E106
S123178090E092BD81BDF89A30B5EFE3F0E0808181FDFDCF85E190E092BD81BDF89A20B51A
S12317A0922F80E0830F911D9C01220F331F880F991F880F991F880F991F280F391F309365
S12317C0360120933501EFE3F0E0808181FDFDCF86E190E092BD81BDF89A30B5EFE3F0E07B
S12317E0808181FDFDCF87E190E092BD81BDF89A20B5922F80E0830F911D90932001809316
S12318001F01EFE3F0E0808181FDFDCF88E190E092BD81BDF89A80B580932301EFE3F0E0B1
S1231820808181FDFDCF89E190E092BD81BDF89A80B580932401EFE3F0E0808181FDFDCF06
S12318408AE190E092BD81BDF89A80B52AE0829FC00111249093260180932501EFE3F0E00F
S1231860808181FDFDCF8BE190E092BD81BDF89A80B52AE0829FC001112490932801809369
S12318802701EFE3F0E0808181FDFDCF8CE190E092BD81BDF89A80B580932B01EFE3F0E01D
S12318A0808181FDFDCF8DE190E092BD81BDF89A80B580932C01EFE3F0E0808181FDFDCF7A
S12318C08EE190E092BD81BDF89A30B5EFE3F0E0808181FDFDCF8FE190E092BD81BDF89A35
S12318E020B5922F80E0830F911D9C01220F331F880F991F880F991F880F991F280F391F12
S123190030932E0120932D01EFE3F0E0808181FDFDCF80E290E092BD81BDF89A30B5EFE35B
S1231920F0E0808181FDFDCF81E290E092BD81BDF89A20B5922F80E0830F911D9C01220F92
S1231940331F880F991F880F991F880F991F280F391F3093300120932F01EFE3F0E080813B
S123196081FDFDCF82E290E092BD81BDF89A30B5EFE3F0E0808181FDFDCF83E290E092BD30
S123198081BDF89A20B5922F80E0830F911D9093320180933101EFE3F0E0808181FDFDCFB5
S12319A084E290E092BD81BDF89A80B52AE0829FC00111249093380180933701EFE3F0E08F
S12319C0808181FDFDCF85E290E092BD81BDF89A80B580933901EFE3F0E0808181FDFDCF53
S12319E086E290E092BD81BDF89A80B52AE0829FC001112490933B0180933A01EFE3F0E047
S1231A00808181FDFDCF87E290E092BD81BDF89A80B52AE0829FC001112490933D018093B5
S1231A203C01EFE3F0E0808181FDFDCF88E290E092BD81BDF89A80B52AE0829FC001112429
S1231A4090933F0180933E01EFE3F0E0808181FDFDCF89E290E092BD81BDF89A80B58E5FC4
S1231A6080934001EFE3F0E0808181FDFDCF8AE290E092BD81BDF89A80B580934101EFE3CA
S1231A80F0E0808181FDFDCF8BE290E092BD81BDF89A80B52AE0829FC001112490932A0187
S1231AA0809329018091290190912A0187399105F8F084E690E090932A018093290120910A
S1231AC0290130912A01EFE3F0E0808181FDFDCF1FBA8BE290E092BD81BDC9016AE070E058
S1231AE00E94223F60BD0FB6F894FA9AF99A0FBEEFE3F0E0808181FDFDCF8CE290E092BD63
S1231B0081BDF89A80B52AE0829FC00111249093430180934201EFE3F0E0808181FDFDCFF1
S1231B208DE290E092BD81BDF89A80B580934401EFE3F0E0808181FDFDCF8EE290E092BDFA
S1231B4081BDF89A80B580931C02EFE3F0E0808181FDFDCF80E390E092BD81BDF89A80B537
S1231B602AE0829FC001112490934A0180934901EFE3F0E0808181FDFDCF82E390E092BD64
S1231B8081BDF89A80B580931B02EFE3F0E0808181FDFDCF83E390E092BD81BDF89A80B5F5
S1231BA080934601EFE3F0E0808181FDFDCF84E390E092BD81BDF89A80B52AE0829FC001C3
S1231BC0112480934501EFE3F0E0808181FDFDCF85E390E092BD81BDF89A80B580934701FF
S1231BE0EFE3F0E0808181FDFDCF86E390E092BD81BDF89A80B580934801EFE3F0E08081C8
S1231C0081FDFDCF87E390E092BD81BDF89A80B580933E05209111013091120180911F012A
S1231C20909120018217930788F4809111019091120120911F0130912001821B930B66E024
S1231C4070E00E94223F60934B0103C089E180934B01EFE3F0E0808181FDFDCF81E390E0A1
S1231C6092BD81BDF89A80B540911501509116012AE0829FC00111244817590788F4EFE3FF
S1231C80F0E0808181FDFDCF1FBA81E390E092BD81BD83E080BD0FB6F894FA9AF99A0FBE06
S1231CA00F2EF4E8CF2EF0E0DF2EF02D84E690E0B6010E941D3C0F2EF6E2EF2EF5E0FF2E50
S1231CC0F02DF7019183808332968F0186E690E0B6010E941D3CF8019183808388E690E000
S1231CE0B6010E941D3CF7013496918380838AE690E0B6010E941D3CF701369691838083E8
S1231D008CE690E0B6010E941D3CF7013896918380838EE690E0B6010E941D3C2AE030E09E
S1231D20E20EF31EF701918380830E949A3A0E94233A12BC11BC1F910F91FF90EF90DF90B2
S1231D40CF9008952F923F924F925F926F927F928F929F92AF92BF92CF92DF92EF92FF9245
S1231D600F931F93DF93CF93CDB7DEB72C970FB6F894DEBF0FBECDBFE4E5F0E08081809367
S1231D80180210820F2EF1E28F2E9924F02DD4011C9204E210E0F80110820F2EF7E2CF2EF5
S1231DA0DD24F02DD6011C920F2EFAE2EF2EFF24F02D8FEFF70180838081806880838081A0
S1231DC0806480830F2EFBE2AF2EBB24F02DD5018C918F778C938C9180648C930E94FD232B
S1231DE00E9493240E94A5000E946D25F8018081816080838081846080838081826080835F
S1231E00808188608083808180618083D7018C91877F8C938C918B7F8C93F40180818062B5
S1231E2080838081806180838C9180618C938C9180628C93D5018C918F7E8C93E5E2F0E0C5
S1231E4080818E7F808380818D7F808380818B7F80838081877F808380818F7E8083F6013D
S1231E60808181608083E8E2F0E080818E7F8083D6018C9182608C9380818D7F80838C91AC
S1231E8084608C9380818B7F80838C9188608C938081877F80838C9180618C938C918062E3
S1231EA08C938C9180648C938C9180688C9380818F7E808380818F7D8083808180648083B2
S1231EC08081806880838CE291E00E94BE2B60934F0170935001809351019093520180E3D3
S1231EE091E00E94BE2B609353017093540180935501909356010E9482070E946D0A789410
S1231F00EAE2F0E080818260808380818E7F80830E94C1378AEA0E941A2681E00E941A26F7
S1231F20809118020E941A2685E50E941A2682E08093230260914F017091500180915101B4
S1231F40909152012DEC3CEC4CEC5EE30E94C93C882384F460914F0170915001809151018F
S1231F60909152012FE832EC45EF5CE30E94183E1816C4F087E19FE9A2E0BDE380934F01F2
S1231F8090935001A0935101B093520180E090ECACE1B1E48093530190935401A093550148
S1231FA0B093560189E060E070E045E050E00E94CB0010921E0210921F02109220021092DD
S1231FC02102E6EAF2E010821182128213823497108211821282138210929C021092A0024D
S1231FE010929F020F2EF4E8CF2EF0E0DF2EF02D84E690E0B6010E941D3C0F2EF6E2EF2ECC
S1232000F5E0FF2EF02DF7019183808332968F0186E690E0B6010E941D3CD80111969C93F9
S12320208E9388E690E0B6010E941D3CF70134969183808380E790E0B6010E941D3CF70191
S123204036969183808382E790E0B6010E941D3CF70138969183808384E790E0B6010E94FD
S12320601D3CEAE0F0E0EE0EFF1ED70111969C938E93A8952DE088E190E00FB6F894A895D0
S1232080809360000FBE20936000E3E3F2E03C96FA83E9830F2EF6ED4F2EF2E05F2EF02D7D
S12320A00F2EF2EA2F2EF2E03F2EF02D91012C5F3F4F3C832B838BE392E008969E838D8383
S12320C0A1E3B2E05096B887AF83E7E2F4E03296FA87E9872BE232E0285F3F4F3C872B8790
S12320E095B1E8E2F0E0990F947080818B7F892B80839081929596959770927080818D7F15
S1232100892B8083A8958091A9019091AA01A091AB01B091AC018158934CA94CB14010F0D7
S12321200E9426060E94043B8091A9019091AA01A091AB01B091AC012091AD013091AE01CB
S12321404091AF015091B001821B930BA40BB50B89589341A040B040F0F08091A90190917D
S1232160AA01A091AB01B091AC018093AD019093AE01A093AF01B093B00180918F02843124
S123218051F4A3E3B2E08D919C91E981FA81608171810E94BC39F20180819181A281B381E7
S12321A00097A105B10509F0BCC080914101882311F04B990AC0AFE3B2E02D913C91809146
S12321C0390190E0281739073CF58091960290919702019690939702809396028091960297
S12321E090919702885B984808F49BC080919502882309F096C081E060E070E040E050E024
S12322000E94CB0081E08093950288EB98E8909397028093960285C0809196029091970240
S12322200197909397028093960280919602909197020B9708F075C080919502813009F017
S123224070C0109295028AE090E0909397028093960280918F028E31B9F56091A901709125
S1232260AA018091AB019091AC01E0901D01F0901E01A0901D01B0901E0160901D0170903C
S12322801E0124E630E040E050E00E94493F00E010E02E0D3F1D401F511F2C5E3F4F4F4F9B
S12322A05F4FCC24DD242A0D3B1D4C1D5D1D88249924260D371D481D591DE6EAF2E02083F9
S12322C03183428353832DC06091A9017091AA018091AB019091AC01E0901D01F0901E01BF
S12322E0A0901D01B0901E0124E630E040E050E00E94493F00E010E02E0D3F1D401F511F63
S12323002C5E3F4F4F4F5F4FCC24DD242A0D3B1D4C1D5D1DA6EAB2E02D933D934D935C9371
S123232013970E94990180918F028E3111F40C94D9198F31A0F48A3009F4B8C48B3038F44D
S1232340882359F1893011F00C948E20CEC0833109F4F6C6843111F00C948E2015C78832E7
S123236011F40C941D1E893250F48F3111F40C94271B803211F00C948E200C948C1B8D33CB
S123238011F40C94441F833611F40C942E208C3311F00C948E200C94D51E84E18093590112
S12323A080935A01E8E2F0E080818E7F808380818D7F808380919C02882351F480919F029F
S12323C09091A002892B21F01092A00210929F028091A9019091AA01A091AB01B091AC0198
S12323E089589341A040B04010F40C94902010929E0210929D0280E060E070E04AE050E033
S12324000E94CB00A1E4B2E02D913C9180912501909126012817390760F088E280938F024D
S123242080912401809359018091240180935A0154C0E3E3F2E080819181883C9105A4F0A4
S123244088E280938F028FE090E09093920280939102109293028091240180935901809143
S1232460240180935A0139C0A3E3B2E08D919C91119787399105C4F0809124018093590114
S12324808091240180935A0189E080938F0210929202109291028D919C9190939902809300
S12324A098021092930219C080912401809359018091240180935A0189E080938F02109278
S12324C092021092910210929302E3E3F2E0808191819093990280939802D1011D921D92B2
S12324E01D921C9213970C94902010921E0210921F021092200210922102EAEDF2E0208129
S12325003181428153818091A9019091AA01A091AB01B091AC0188519C4FAF4FBF4F28170D
S123252039074A075B07B0F4F10180819181A281B3810297A105B10568F0A3E3B2E08D9121
S12325409C9145973CF082E060E070E048EE53E00E94CB00EEEDF2E080819181A281B38163
S12325600097A105B10509F074C08091910290919202889708F06DC08091240180935901F7
S12325808091240180935A014091190250911A0283E060E070E00E94CB0080919C028F5FAD
S12325A080939C0280919102909192028A96909392028093910280913A0190913B019093C4
S12325C01A018093190180919C028230A8F0EFE3F0E0808181FDFDCF81E390E092BD81BD68
S12325E0F89A40B58AE0489FA001112481E060E070E00E94CB0009C0409115015091160123
S123260081E060E070E00E94CB00F10180819181A281B3810196A11DB11D80839183A2839D
S1232620B3836091A9017091AA018091AB019091AC0124E630E040E050E00E94493F822F49
S1232640932FA42FB52FEB81FC8180839183A283B383EEEDF2E080819181A281B3810097F4
S1232660A105B10509F070C0F10180819181A281B3810197A105B10509F066C0F20180816E
S12326809181A281B3810097A105B10509F05CC0A3E3B2E08D919C919093990280939802F7
S12326A0409113015091140183E060E070E00E94CB0080911301909114012091910230917B
S12326C092026AE070E00E94223F620F731F709392026093910284E060E070E040EB54E052
S12326E00E94CB0081E090E090939E0280939D02F10180819181A281B3810196A11DB11DA4
S123270080839183A283B3836091A9017091AA018091AB019091AC0124E630E040E050E007
S12327200E94493F822F932FA42FB52FEB81FC8180839183A283B383809124018093590143
S12327408091240180935A018091980290919902A3E3B2E02D913C91449628173907E0F09E
S123276088EE93E09093990280939802809124012091230190E0820F911D959587958093EE
S12327805901809124012091230190E0820F911D9595879580935A01EEEDF2E080819181AD
S12327A0A281B3810097A105B105A1F5F10180819181A281B3810297A105B10558F180918A
S12327C01C0290E00496880F991FEBE2F2E0E80FF91F4081518180914201909143012091D3
S12327E04401821B910948175907A0F480911B02813039F480E060E070E044E150E00E9413
S1232800CB00409113015091140183E064E170E00E94CB00A2EEB2E02D913D914D915C9130
S12328208091A9019091AA01A091AB01B091AC0188519C4FAF4FBF4F281739074A075B0740
S1232840B0F480919D0290919E02059780F484E060E070E040EB54E00E94CB0080919D02DF
S123286090919E02019690939E0280939D02E2EEF2E080819181A281B3810097A105B10588
S1232880C1F4A3E3B2E02D913C9180912101909122018217930768F484E060E070E048EBAF
S12328A05BE00E94CB008AE090E090939E0280939D02F10180819181A281B3810297A10582
S12328C0B10508F4CFC020813181428153818091400190E0A0E0B0E0281739074A075B07C5
S12328E008F0C0C0F20180819181A281B3810097A105B10509F0B6C0A3E3B2E0ED90FC907C
S1232900F101608171818281938100912101109122010253104029E130E040E050E00E94AF
S1232920F73E060F171F0E151F0508F09BC06091A9017091AA018091AB019091AC01A6EA17
S1232940B2E0ED90FD900D911C9124E630E040E050E00E94493F2E193F09400B510B23336C
S123296031054105510508F47DC06091A9017091AA018091AB019091AC01E6EAF2E0E08074
S1232980F1800281138124E630E040E050E00E94493FE216F3060407150708F063C0AFE352
S12329A0B2E02D913C9180915701909158012817390708F057C084E060E070E040E157E237
S12329C00E94CB006091190170911A01409117015091180181E00E94CB00F10180819181A9
S12329E0A281B3810196A11DB11D80839183A283B3836091A9017091AA018091AB019091C2
S1232A00AC01E0901901F0901A01A0901701B090180100E010E024E630E040E050E00E9463
S1232A20493FE20EF31E041F151FCC24DD24EA0CFB1C0C1D1D1DAB81BC81ED92FD920D933A
S1232A401C931397809137019091380190931A018093190180912301809359018091230134
S1232A6080935A01F10120813181428153818091400190E0A0E0B0E0281739074A075B0704
S1232A8008F462C0F20180819181A281B3810097A105B10509F058C0A3E3B2E02D913C9110
S1232AA080913C0190913D0182179307E0F4EFE3F2E0208131818091570190915801281745
S1232AC0390788F4D1011D921D921D921C9213978AE080938F0282E060E070E040ED57E09B
S1232AE00E94CB0031C06091A9017091AA018091AB019091AC01E6EAF2E0E080F1800281AC
S1232B00138124E630E040E050E00E94493F80EB94E0A0E0B0E0E80EF91E0A1F1B1FE21632
S1232B20F3060407150780F4D1011D921D921D921C9213978AE080938F0282E060E070E0C6
S1232B404AE050E00E94CB00EEEDF2E080819181A281B3810097A105B105D1F080911C02B0
S1232B6090E00496880F991FEBE2F2E0E80FF91F208131818091420190914301821793070B
S1232B8038F483E060E070E040E050E00E94CB00EEEDF2E080819181A281B3810097A10501
S1232BA0B10549F5F10180819181A281B3810297A105B10500F180911C0290E00496880F0B
S1232BC0991FEBE2F2E0E80FF91F40815181809142019091430120914401821B91094817B3
S1232BE0590748F4409113015091140183E060E070E00E94CB00F10180819181A281B3819E
S1232C000297A105B10570F1E2EEF2E080819181A281B3810097A105B10521F580919D0295
S1232C2090919E020597F0F0A3E3B2E08D919C91883C9105BCF480919C02823048F41092A7
S1232C408F0281E090E09093A00280939F020AC084E060E070E048E853E10E94CB0083E69D
S1232C6080938F02E1E4F2E02081318180912501909126018C599F4F2817390710F40C944D
S1232C80902088E280938F02A3E3B2E08D919C91909399028093980280919802909199023D
S1232CA090939B0280939A020C94902010921E0210921F021092200210922102A895109264
S1232CC0A00210929F0210929C02EEEDF2E080819181A281B3810097A105B105D1F08091EF
S1232CE01C0290E00496880F991FEBE2F2E0E80FF91F208131818091420190914301821706
S1232D00930738F483E060E070E040E050E00E94CB00AAEDB2E02D913D914D915C918091A8
S1232D20A9019091AA01A091AB01B091AC0188519C4FAF4FBF4F281739074A075B0780F4D8
S1232D40F10180819181A281B3810097A105B10539F482E060E070E040ED57E00E94CB0030
S1232D60E2EDF2E080819181A281B3810097A105B105A1F4F10180819181A281B3810097C9
S1232D80A105B10559F06091350170913601409133015091340180E00E94CB00809123010E
S1232DA080935A018091230180935901A2EEB2E02D913D914D915C918091A9019091AA01FF
S1232DC0A091AB01B091AC0188519C4FAF4FBF4F281739074A075B0738F484E060E070E002
S1232DE048EE53E00E94CB00F20180819181A281B3810097A105B10509F0AFC0F10180814E
S1232E009181A281B3810097A105B10509F0A5C06091A9017091AA018091AB019091AC0122
S1232E20A6EAB2E0ED90FD900D911C9124E630E040E050E00E94493FE216F306040715076B
S1232E4008F08BC06091A9017091AA018091AB019091AC01E6EAF2E0A080B180C280D380D1
S1232E60E0903E01F0903F0124E630E040E050E00E94493F2A193B094C095D0900E010E039
S1232E80E216F3060407150708F067C0A3E3B2E0AD90BC90E0901F01F090200160914B01E8
S1232EA0F1012081318142815381CC24B7FCC094DC2C70E080E090E00E94F73E00E010E06C
S1232EC06E0D7F1D801F911F6A157B058C059D0508F000C1AFE3B2E02D913C918091570185
S1232EE0909158012817390708F0F4C040911B0150911C0181E060E070E00E94CB0040910F
S1232F00490150914A0182E060E070E00E94CB00F10180819181A281B3810196A11DB11D59
S1232F2080839183A283B3836091A9017091AA018091AB019091AC0124E630E040E050E0DF
S1232F400E94493F822F932FA42FB52FEB81FC8180839183A283B383BDC0F201808191813B
S1232F60A281B3810097A105B10509F0B3C0F10180819181A281B3810097A105B10509F44B
S1232F80A9C06091A9017091AA018091AB019091AC01A6EAB2E0ED90FD900D911C9124E671
S1232FA030E040E050E00E94493FE216F3060407150708F08FC06091A9017091AA018091CC
S1232FC0AB019091AC01E6EAF2E0A080B180C280D38080901D0190901E01E0901B01F09072
S1232FE01C0124E630E040E050E00E94493F2A193B094C095D09E80CF91C00E010E0E21609
S1233000F3060407150708F065C0A3E3B2E0AD90BC90E0901F01F090200160914B01F1016E
S12330202081318142815381CC24B7FCC094DC2C70E080E090E00E94F73E00E010E06E0D61
S12330407F1D801F911F6A157B058C059D0508F041C0AFE3B2E02D913C918091570190911D
S1233060580128173907B0F540911B0150911C0181E060E070E00E94CB004091490150918A
S12330804A0182E060E070E00E94CB00F10180819181A281B3810196A11DB11D80839183EC
S12330A0A283B3836091A9017091AA018091AB019091AC0124E630E040E050E00E94493F4B
S12330C0822F932FA42FB52FEB81FC8180839183A283B383F10180819181A281B381029772
S12330E0A105B10518F083E180938F02A3E3B2E08D919C918436910514F410928F02E1E4AD
S1233100F2E02081318180912501909126012817390710F40C9490208EE180938F02A3E39B
S1233120B2E08D919C919093990280939802809198029091990290939B0280939A02F0C7B6
S123314084E180938F02F10110821182128213820E946D0AE8E2F0E0808181608083808189
S123316082608083109292021092910210929C0210921E0210921F021092200210922102AD
S12331808081877F8083CCC78091230180935A0180912301809359010E947705E2EDF2E08A
S12331A080819181A281B3810097A105B10559F460913501709136014091330150913401E7
S12331C080E00E94CB00A2EEB2E02D913D914D915C918091A9019091AA01A091AB01B09100
S12331E0AC0188519C4FAF4FBF4F281739074A075B0738F484E060E070E040EB54E00E94FB
S1233200CB00F20180819181A281B3810097A105B10509F0B2C06091A9017091AA018091CC
S1233220AB019091AC01A6EAB2E0ED90FD900D911C9124E630E040E050E00E94493FE2160D
S1233240F3060407150708F098C06091A9017091AA018091AB019091AC01E6EAF2E0A08066
S1233260B180C280D38080901D0190901E01E0901B01F0901C0124E630E040E050E00E94E2
S1233280493F2A193B094C095D09E80CF91C00E010E0E216F306040715070CF06EC0A7E2BC
S12332A0B4E02D913C9180911101909112018217930708F062C0EFE3F2E02081318180913F
S12332C05701909158012817390708F056C080911D02882331F080911D02815080931D025C
S12332E009C040911B0150911C0181E060E070E00E94CB00A3E3B2E08D919C919093990297
S123330080939802809194028F5F80939402F10180819181A281B3810196A11DB11D80833C
S12333209183A283B3836091A9017091AA018091AB019091AC0124E630E040E050E00E943C
S1233340493F822F932FA42FB52FEB81FC8180839183A283B3834091490150914A0182E0B3
S123336060E070E00E94CB008091A102813029F48EE180938F021092A102A1E4B2E02D919D
S12333803C9180912501909126012817390720F081E08093A10202C01092A102E3E3F2E098
S12333A080819181843691050CF0BAC610928F02B7C610921E0210921F021092200210928F
S12333C02102A3E3B2E02D913C91119780919A0290919B028217930730F48D919C9190934B
S12333E09B0280939A0210929C0280912B018093590180912B0180935A0180919A0290911A
S12334009B028752924038F0E3E3F2E080819181C2970CF4D6C0A2EEB2E02D913D914D9112
S12334205C918091A9019091AA01A091AB01B091AC0188519C4FAF4FBF4F281739074A07A9
S12334405B0738F484E060E070E040EB54E00E94CB00E2EDF2E080819181A281B381009778
S1233460A105B10559F46091350170913601409133015091340180E00E94CB00F201808164
S12334809181A281B3810097A105B10509F099C06091A9017091AA018091AB019091AC01A8
S12334A0A6EAB2E0ED90FD900D911C9124E630E040E050E00E94493FE216F30604071507E5
S12334C008F07FC06091A9017091AA018091AB019091AC01E6EAF2E0A080B180C280D38057
S12334E080902F0190903001E0902D01F0902E0124E630E040E050E00E94493F2A193B09CF
S12335004C095D09E80CF91C00E010E0E216F306040715070CF055C0A7E2B4E02D913C9142
S123352080913101909132018217930708F049C0EFE3F2E0208131818091570190915801E2
S123354028173907F0F540912D0150912E0181E060E070E00E94CB004091490150914A014F
S123356082E060E070E00E94CB00A3E3B2E08D919C919093990280939802F1018081918115
S1233580A281B3810196A11DB11D80839183A283B3836091A9017091AA018091AB01909116
S12335A0AC0124E630E040E050E00E94493F822F932FA42FB52FEB81FC8180839183A28377
S12335C0B383A1E4B2E08D919C9120912501309126014091270150912801241B350B821775
S12335E09307F8F4E3E3F2E080819181803991051CF410928F0215C0D1011D921D921D9250
S12336001C92139780E280938F0210929902109298028091240180935901809124018093E3
S12336205A01E1E4F2E04081518120912501309126018091290190912A01820F931F8417DD
S1233640950708F06DC588E280938F0269C580912B018093590180912B0180935A01AAED78
S1233660B2E02D913D914D915C918091A9019091AA01A091AB01B091AC0188519C4FAF4F49
S1233680BF4F281739074A075B0738F482E060E070E048E552E00E94CB00E2EEF2E02081B9
S12336A03181428153818091A9019091AA01A091AB01B091AC0188519C4FAF4FBF4F28175C
S12336C039074A075B0738F484E060E070E040EB54E00E94CB006091A9017091AA018091AF
S12336E0AB019091AC01E0908B02F0908C0200918D0210918E0224E630E040E050E00E94E4
S1233700493FE216F3060407150708F009C510928F0210929C0204C5AAEDB2E02D913D914E
S12337204D915C918091A9019091AA01A091AB01B091AC0188519C4FAF4FBF4F2817390719
S12337404A075B0760F4F10180819181A281B38182E060E070E040ED57E00E94CB00A2EEAF
S1233760B2E02D913D914D915C918091A9019091AA01A091AB01B091AC0188519C4FAF4F48
S1233780BF4F281739074A075B0738F484E060E070E040EB54E00E94CB00F10180819181F4
S12337A0A281B3810097A105B10509F081C0F20180819181A281B3810097A105B10509F038
S12337C077C0409113015091140183E060E070E00E94CB004091450181E06CE370E050E02C
S12337E00E94CB00F10180819181A281B3810196A11DB11D80839183A283B3836091A901CC
S12338007091AA018091AB019091AC01E0901D01F0901E0124E630E040E050E00E94493FAC
S123382089019A01C70165E070E00E94223F660F771F660F771F80E090E0601771078207A1
S1233840930758F56091A9017091AA018091AB019091AC01E0901D01F0901E0124E630E064
S123386040E050E00E94493F89019A01C70165E070E00E94223F660F771F660F771F80E0CF
S123388090E0061B170B280B390BA6EAB2E00D931D932D933C9313972BC082E390E0A0E00F
S12338A0B0E0E6EAF2E080839183A283B38320C0F10180819181A281B3810197A105B10530
S12338C0B9F4F20180819181A281B3810097A105B10571F48091980290919902892B41F432
S12338E0A3E3B2E08D919C919093990280939802E3E3F2E0208131818091980290919902A4
S12339008C599F4F28173907F0F48091980290919902892BC1F080819181805991409CF454
S1233920EEEDF2E080819181A281B3810097A105B10549F4409113015091140183E060E0BE
S123394070E00E94CB00EEEDF2E080819181A281B3810097A105B10571F0A3E3B2E08D9105
S12339609C91875292403CF083E060E070E040E050E00E94CB00E3E3F2E020813181809193
S12339809802909199028C599F4F8217930730F48091980290919902892B41F4A3E3B2E03B
S12339A08D919C91875292400CF4F3C0EEEDF2E080819181A281B3810097A105B10539F027
S12339C083E060E070E040E050E00E94CB0084E690E09093990280939802809123018093A6
S12339E059018091230180935A01F10180819181A281B3810097A105B10509F4CAC020814F
S1233A003181428153818091460190E00296AA2797FDA095BA2F281739074A075B0708F04C
S1233A20B8C0F20180819181A281B3810097A105B10509F0AEC0A3E3B2E0ED90FC90F10140
S1233A40608171818281938100912101109122010951104029E130E040E050E00E94F73E16
S1233A60060F171F0E151F0508F093C06091A9017091AA018091AB019091AC01A6EAB2E071
S1233A80ED90FD900D911C9124E630E040E050E00E94493F2E193F09400B510B2333310577
S1233AA04105510508F475C06091A9017091AA018091AB019091AC01E6EAF2E0E080F180F0
S1233AC00281138124E630E040E050E00E94493FE216F3060407150708F05BC0AFE3B2E0E8
S1233AE02D913C9180915701909158012817390708F04FC084E060E070E040E157E20E94DE
S1233B00CB006091190170911A01409117015091180181E00E94CB00F10180819181A281D6
S1233B20B3810196A11DB11D80839183A283B3836091A9017091AA018091AB019091AC01E6
S1233B40E0901901F0901A01A0901701B090180100E010E024E630E040E050E00E94493F37
S1233B60E20EF31E041F151FCC24DD24EA0CFB1C0C1D1D1DAB81BC81ED92FD920D931C93C2
S1233B801397809137019091380190931A0180931901F1012081318142815381809140013B
S1233BA090E0A0E0B0E0281739074A075B0750F1F20180819181A281B3810097A105B105BE
S1233BC009F5A3E3B2E02D913C9180913C0190913D0182179307B0F4F10110821182128211
S1233BE013828AE080938F02EB81FC8180819181A281B38180559040A040B040808391833F
S1233C00A283B383A3E3B2E08D919C918436910524F410929C0210928F02E1E4F2E02081CF
S1233C20318180912501909126018217930708F077C28EE180938F0273C210921E0210923F
S1233C401F02109220021092210280912C018093590180912C0180935A01F2018081918159
S1233C60A281B3810097A105B10539F081E060E070E040E050E00E94CB00A3E3B2E08D91E9
S1233C809C918059914044F080912301809359018091230180935A01E3E3F2E08081918125
S1233CA0883C91050CF46AC0A2EEB2E02D913D914D915C918091A9019091AA01A091AB019F
S1233CC0B091AC0188519C4FAF4FBF4F281739074A075B0738F484E060E070E040EB54E071
S1233CE00E94CB00E2EDF2E080819181A281B3810097A105B10591F4809135019091360131
S1233D004091330150913401BC01660F771F680F791F7695679580E00E94CB00A1E4B2E0C2
S1233D208D919C9120912501309126014091270150912801241B350B8217930708F0F0C117
S1233D40E3E3F2E080819181805991400CF0E8C1D1011D921D921D921C92139780E28093B9
S1233D608F02109299021092980280912401809359018091240180935A01D2C1E1E4F2E0C4
S1233D808081918120912501309126014091270150912801241B350B8217930708F0C0C11F
S1233DA010928F0210929C02BBC18091230180935A018091230180935901E2EDF2E0808129
S1233DC09181A281B3810097A105B10559F46091350170913601409133015091340180E05C
S1233DE00E94CB00A2EEB2E02D913D914D915C918091A9019091AA01A091AB01B091AC0187
S1233E0088519C4FAF4FBF4F281739074A075B0738F484E060E070E040EB54E00E94CB00B0
S1233E20E3E3F2E02081318180919A0290919B028217930730F48081918190939B028093EB
S1233E409A02A3E3B2E02D913C91119780919A0290919B02865990402817390728F08D91A8
S1233E609C918F5E92402CF0109294028DE380938F02E3E3F2E080819181843691050CF0F3
S1233E804FC110928F024CC1E2EDF2E080819181A281B3810097A105B10559F4609135015C
S1233EA070913601409133015091340180E00E94CB00A2EEB2E02D913D914D915C91809154
S1233EC0A9019091AA01A091AB01B091AC0188519C4FAF4FBF4F281739074A075B0738F46F
S1233EE084E060E070E040EB54E00E94CB00F20180819181A281B3810097A105B10509F0B5
S1233F008BC06091A9017091AA018091AB019091AC01A6EAB2E0ED90FD900D911C9124E6FF
S1233F2030E040E050E00E94493FE216F3060407150708F071C06091A9017091AA0180915A
S1233F40AB019091AC01E6EAF2E0A080B180C280D380E0901D01F0901E0180901B019090E2
S1233F601C0124E630E040E050E00E94493F2A193B094C095D09EE0CFF1CE80CF91C00E04C
S1233F8010E0E216F3060407150708F045C0A3E3B2E02D913C918091110190911201821785
S1233FA09307D0F540911B0150911C0181E060E070E00E94CB00E3E3F2E080819181909387
S1233FC0990280939802809194028F5F80939402F10180819181A281B3810196A11DB11DD8
S1233FE080839183A283B3836091A9017091AA018091AB019091AC0124E630E040E050E00F
S12340000E94493F822F932FA42FB52FEB81FC8180839183A283B38380919402843028F07A
S12340201092940283E180938F02A1E4B2E02D913C9180912501909126018217930718F4DC
S12340408EE180938F02E3E3F2E080819181843691050CF065C010928F0262C080912401A2
S1234060809359018091240180935A01EEEDF2E080819181A281B3810097A105B10539F0F8
S123408083E060E070E040E050E00E94CB00F20180819181A281B3810097A105B10539F0F3
S12340A081E060E070E040E050E00E94CB00EAEDF2E080819181A281B3810097A105B10548
S12340C039F082E060E070E040E050E00E94CB00E2EDF2E080819181A281B3810097A105BC
S12340E0B10539F080E060E070E040E050E00E94CB00439907C084E060E070E040EB54E03A
S12341000E94CB0082E090E09093A00280939F02E8E2F0E080818860808302C010928F0268
S123412080910203883398F01092020383E193E00E94542783E993E00E9454278091FE027A
S12341409091FF0201969093FF028093FE02A8950E94F637882309F46DC080918F02409117
S1234160A9015091AA016091AB017091AC012BE232E00E940D3881E080932302AB85BC85AA
S12341806D917C91882777FD8095982F0E94683D6093CB037093CC038093CD039093CE0360
S12341A080917C008630F1F40E9408388823D1F0809178009091790060E00E9401036AE032
S12341C070E00E94363F862F972FEDE2F2E091838083808191818B3591053CF083E6809330
S12341E08F0203C086E080937C00E3E3F2E080819181A7E2B4E011969C938E93E985FA85C6
S1234200208131818D919C911197820F931F9695879591838083FD01349620813181A9856A
S1234220BA858D919C91820F931F9695879591838083DDC280912402813009F0D8C2109293
S1234240240280912302843009F0B5C080913E05813081F50F2EF9E58F2EF2E09F2EF02DCD
S1234260F4016081718182819381E0907800F090790026E636E646E65FE30E94613E5B0147
S12342806C0100E010E0C801B7010E94663D23E938E144E05EE30E94613E9B01AC01C6013C
S12342A0B5010E94653CD4016D937D938D939C9313972FC00F2EF9E58F2EF2E09F2EF02DA0
S12342C0F4016081718182819381E0907800F090790026E636E646E65FE30E94613E5B01E7
S12342E06C0100E010E0C801B7010E94663D20E932EC45EF5DE30E94613E9B01AC01C601CB
S1234300B5010E94653CD4016D937D938D939C9313976091590270915A0280915B0290918A
S12343205C020E94353DE3E3F2E07183608380819181A7E2B4E011969C938E93E985FA8584
S1234340208131818D919C911197820F931F9695879591838083FD01349620813181A98529
S1234360BA858D919C91820F931F969587959183808311E01093230210932302E3E3F2E0F5
S123438060817181882777FD8095982F0E94683D6093CB037093CC038093CD039093CE0396
S12343A0E2E2F0E080818F7D808380818F7E808310937C001CC280912302813041F486E0C5
S12343C0809323020E94043B10927C0010C280912302853009F046C00F2EFDE58F2EF2E038
S12343E09F2EF02DD4016D917D918D919C91E0907800F09079002DEC3CEC4CE45FE30E946D
S1234400613E5B016C0100E010E0C801B7010E94663D20E932EC45E75EE30E94613E9B0129
S1234420AC01C601B5010E94653CF401608371838283938360817181828193810E943A3D21
S1234440709336026093350292E090932302E2E2F0E08081806280838081806180839093B7
S12344607C00C5C180912302823019F5AFE3B2E02D913C9111974091780050917900C9017C
S1234480880F991F880F991F880F991F821B930B840F951F969587959695879596958795D4
S12344A011969C938E9387E08093230210927C009EC180912302863071F410922302E2E209
S12344C0F0E080818062808380818F7E808383E080937C008CC180912302882309F085C0B3
S12344E00F2EF9E48F2EF2E09F2EF02DF4016081718182819381E0907800F090790023E35F
S123450033E343E75FE30E94613E5B016C0100E010E0C801B7010E94663D2DEC3CEC4CE404
S12345205DE30E94613E9B01AC01C601B5010E94653CD4016D937D938D939C9313976D9111
S12345407D918D919C910E943A3DEBE2F2E07183608385E08093230260817181E0904F013F
S1234560F09050010091510110915201882777FD8095982F0E94683DA80197010E94613EC7
S1234580609385027093860280938702909388026091850270918602809187029091880283
S12345A0209153013091540140915501509156010E94643C6093850270938602809387029A
S12345C0909388028091850290918602A0918702B091880280934B0390934C03A0934D030E
S12345E0B0934E0310927C0002C180912302873009F043C0A5E6B2E06D917D918D919C91E5
S1234600E0907800F090790026E636E646E65FE30E94613E5B016C0100E010E0C801B701C4
S12346200E94663D20E932EC45EF5DE30E94613E9B01AC01C601B5010E94653CE5E6F2E0AF
S1234640608371838283938360817181828193810E94353D70933A026093390283E0809383
S12346602302E2E2F0E080818F7D808380818061808386E080937C00BAC080912302833030
S123468009F052C0A5E5B2E06D917D918D919C91E0907800F090790026E636E646E65FE321
S12346A00E94613E5B016C0100E010E0C801B7010E94663D2DEC3CEC4CEC5DE30E94613E5C
S12346C09B01AC01C601B5010E94653CE5E5F2E06083718382839383608171818281938155
S12346E00E943A3DA1E3B2E011967C936E9388E0809323028D919C9160E00E940103EF818F
S1234700F88591838083808191816AE070E00E94363F862F972FE1E3F2E03C969183808343
S123472087E080937C0063C080912302883009F058C0A9E6B2E06D917D918D919C910F2EA8
S1234740F8E78F2E9924F02DF401E080F1802DEC3CEC4CE45FE30E94613E5B016C0100E07C
S123476010E0C801B7010E94663D2DEC3CEC4CE45EE30E94613E9B01AC01C601B5010E9424
S1234780653CA9E6B2E06D937D938D939C931397EBE3F2E020813181D4014D915C91C901ED
S12347A0880F991F880F991F880F991F821B930B840F951F969587959695879596958795B1
S12347C09183808384E0809323028081918161E00E940103ED81FE819183808310927C0006
S12347E006C0109223028091230280937C000E94E2030E94B0030C947010E5E4F0E010823C
S1234800AEE6B0E08C9183608C9380818360808317BCEAE2F0E08081806180838081806233
S12348208083EBE2F0E080818F7E808380818F7D808308951F920F920FB60F9211245F9337
S12348406F937F938F939F93AF93BF93EF93FF93F894EBE2F0E08081806180838081806253
S12348608083809101038F5F80930103809101038734F0F01092010390915A0189E1989FA4
S1234880C00111246AE070E00E94223F6B5F87B5861730F4E7E4F0E080818F5F808308C065
S12348A087B5681728F4E7E4F0E08081815080837894FF91EF91BF91AF919F918F917F91A1
S12348C06F915F910F900FBE0F901F9018951F920F920FB60F9211248F939F93AF93BF93A8
S12348E0EF93FF93F8948091E2029091E302A091E402B091E5020097A105B10541F0EBE2E9
S1234900F0E080818F7D808380818F7E80837894FF91EF91BF91AF919F918F910F900FBE3A
S12349200F901F901895E1EBF0E01082A0E7B0E08C9181608C9380818760808381E08093B7
S1234940B20008951F920F920FB60F9211248F939F93AF93BF9381E0809324028091A901DA
S12349609091AA01A091AB01B091AC014296A11DB11D8093A9019093AA01A093AB01B0938B
S1234980AC01809102038F5F80930203BF91AF919F918F910F900FBE0F901F9018951F9252
S12349A00F920FB60F9211248F939F93EF93FF9380910003813051F410920003E8E8F0E000
S12349C0808191818C599F4F91838083FF91EF919F918F910F900FBE0F901F9018951F925E
S12349E00F920FB60F9211240F900FBE0F901F9018951F920F920FB60F9211240F900FBEB7
S1234A000F901F9018951F920F920FB60F9211240F900FBE0F901F9018951F920F920FB62C
S1234A200F9211242F933F935F936F937F938F939F93AF93BF93EF93FF93E4E8F0E02081C9
S1234A403181118210828091CF019091D001880F991F880F991F820F931F880F991F6AE02E
S1234A6070E00E94223F862F972F9093D0018093CF01FF91EF91BF91AF919F918F917F918D
S1234A806F915F913F912F910F900FBE0F901F9018951092800088E893E190938900809366
S1234AA0880080E197E290938B0080938A00E1E8F0E080E8808383E08083EFE6F0E0808135
S1234AC081608083E9E6F0E080818A608083EDE3F0E0808183608083089588E98093C100F8
S1234AE08FE08093C4008BEA95E09093770580937605909373058093720589E795E0909328
S1234B007505809374059093DE058093DD05109278051092240508951F920F920FB60F9251
S1234B2011248F939F93EF93FF9380917805882311F1E0917605F091770581918093C600C5
S1234B40F0937705E0937605ED5DF54030F08BEA95E090937705809376058091780581504F
S1234B608093780580917805882329F4E1ECF0E080818F7D8083FF91EF919F918F910F909F
S1234B800FBE0F901F9018951F920F920FB60F9211242F938F939F93EF93FF938091C6005B
S1234BA0E091DD05F091DE058083809124058F5F809324058091DD059091DE050196909322
S1234BC0DE058093DD058B5A954030F089E795E09093DE058093DD05FF91EF919F918F91DF
S1234BE02F910F900FBE0F901F90189580912405882319F42FEF3FEF1AC0F89480912405AC
S1234C00815080932405E0917405F09175052191F0937505E0937405EB5AF54030F089E7F9
S1234C2095E09093750580937405789430E0822F932F0895982F80917805823310F080E03C
S1234C400895F894809178058F5F80937805E0917205F09173059083809172059091730506
S1234C60019690937305809372058D5D954030F08BEA95E09093730580937205E1ECF0E0E9
S1234C80808180628083789481E00895CF93DF93EC0104C00E941A268111219688818823BC
S1234CA0C9F781E0DF91CF91089589ED91E00E94462608958091240508958F929F92AF9266
S1234CC0BF92CF92DF92EF92FF920F931F93DF93CF93CDB7DEB729970FB6F894DEBF0FBEDF
S1234CE0CDBF8C01F62EE42EDE011196ECEDF1E089E001900D928150E1F749E00F2EF9E0B0
S1234D00AF2EBB24F02D6E010894C11CD11C0F2EFEE28F2EF02D9924FF2071F09501241BD8
S1234D2031098F2D90E02817390730F04150F601E40FF11D8082F92C4150F601E40FF11D31
S1234D40C8016AE070E00E94223F805D8083C8016AE070E00E94223F862F972F8C01011585
S1234D60110511F4FF2019F085E08F15A8F689E0182F1E19193068F47E010894E11CF11C94
S1234D80F701E10FF11D80810E941A261F5F1930B8F329960FB6F894DEBF0FBECDBFCF915E
S1234DA0DF911F910F91FF90EF90DF90CF90BF90AF909F908F900895EF92FF920F931F9374
S1234DC0FC018C010F5F1F4F80810E941A2678010894E11CF11CF80180810E941A26F70193
S1234DE080810E941A26F70181810E941A261F910F91FF90EF900895282F392FEFE3F0E094
S1234E00808181FDFDCF822F932F92BD81BDF89A80B50895262F372FA901BA016F5F7F4F23
S1234E20DC019D91EFE3F0E0808181FDFDCF1FBA52BD41BD90BD0FB6F894FA9AF99A0FBEFE
S1234E40AB014F5F5F4F2D91EFE3F0E0808181FDFDCF1FBA72BD61BD20BD0FB6F894FA9AB3
S1234E60F99A0FBE2C91EFE3F0E0808181FDFDCF1FBA52BD41BD20BD0FB6F894FA9AF99AE9
S1234E800FBE11962C91EFE3F0E0808181FDFDCF1FBACA01019692BD81BD20BD0FB6F894FA
S1234EA0FA9AF99A0FBE08952F923F924F925F926F927F928F929F92AF92BF92CF92DF9231
S1234EC0EF92FF920F931F93DF93CF93CDB7DEB762970FB6F894DEBF0FBECDBF9A8B898B02
S1234EE0DC011C966D917D918D919C911F97FD01E059FF4F20813181428153810E94643C61
S1234F0020E030E040E050E00E94C93C882309F450C0E989FA89E85BFF4FFA87E987A08037
S1234F20B180C280D380AD82BE82CF82D886E989FA896485758586859785E059FF4F208162
S1234F40318142815381A989BA899496ED90FD900D911C9197971896AD90BD90CD90DC90E1
S1234F601B97D8962D903D904D905C90DB970E94643C3B014C01C801B701A60195010E941D
S1234F80613EA20191010E94643C9B01AC01C401B3010E94613E9B01AC016D817E818F81AE
S1234FA098850E94643CE985FA856083718382839383A989BA891C96AD90BD90CD90DC9035
S1234FC01F9794966D917D918D919C91979718962D913D914D915C911B97D896ED90FD9039
S1234FE00D911C91DB970E94613EA80197010E94643C9B01AC01C601B5010E94613EE989B3
S1235000FA89EC5BFF4FFC87EB876083718382839383E989FA89E459FF4F60817181828137
S12350209381E989FA89E45BFF4FFE87ED872081318142815381E989FA89E859FF4F2080CF
S1235040318042805380A989BA89D896AD90BD90CD90DC90DB97FD01E45AFF4FE080F18003
S1235060028113810E94613E3B014C01C601B501A80197010E94643C9B01AC01C201B1018D
S12350800E94613E9B01AC01C401B3010E94643CED85FE856083718382839383AB85BC856F
S12350A06D917D918D919C91E989FA89E85BFF4F2081318142815381ED85FE85E080F1805F
S12350C0028113810E94653CA80197010E94653CE989FA89E85AFF4F608371838283938377
S12350E0A989BA898C91882309F45FC0A85BBF4FB88BAF872D903D904D905C90E989FA8981
S1235100E05AFF4FE080F18002811381E989FA89608571858285938520AD31AD42AD53AD92
S1235120EC59FF4FA080B180C280D380A982BA82CB82DC82E989FA89EC5AFF4F6080718086
S123514082809380E989FA89E85AFF4FA080B180C280D3800E94643C9B01AC01C801B701BF
S12351600E94613E9B01AC01C201B1010E94653C7B018C01C401B301A60195010E94643CE8
S12351809B01AC0169817A818B819C810E94613E9B01AC01C801B7010E94653CAF85B889F1
S12351A06D937D938D939C931397E989FA898481813009F07DC0E85AFF4F2081318142815B
S12351C05381A989BA899896ED90FD900D911C919B9760E070E088EC92E40E94643CA80168
S12351E097010E94C93C88236CF4E989FA8980A591A5A2A5B3A5EC5AFF4F80839183A283A2
S1235200B3833FC0E989FA89E85AFF4F2081318142815381A989BA899C96ED90FD900D9197
S12352201C919F9760E070E088EC92E40E94643CA80197010E94183E18166CF4E989FA890F
S123524084A595A5A6A5B7A5EC5AFF4F80839183A283B38316C0E989FA89E85AFF4F20813E
S123526031814281538160E070E088EC92E40E94643CE989FA89EC5AFF4F608371838283C0
S12352809383E989FA89EC5AFF4F608171818281938126E636ED43E254E40E94613E0E9412
S12352A03A3DE989FA89E458FF4F7183608368C0E989FA89E85AFF4F608171818281938186
S12352C0A989BA8998962D913D914D915C919B970E94C93C88236CF4E989FA8980A591A59C
S12352E0A2A5B3A5EC5AFF4F80839183A283B38331C0E989FA89E85AFF4F608171818281B9
S12353009381A989BA899C962D913D914D915C919F970E94183E18166CF4E989FA8984A59D
S123532095A5A6A5B7A5EC5AFF4F80839183A283B38310C0E989FA89E85AFF4F808191811A
S1235340A281B381E989FA89EC5AFF4F80839183A283B383E989FA89EC5AFF4F608171819B
S12353608281938120E030E04BE154E40E94613E0E943A3DE989FA89E458FF4F71836083EE
S1235380E989FA8980AD91ADA2ADB3ADE45AFF4F80839183A283B383E989FA8984859585E4
S12353A0A685B785E059FF4F80839183A283B383A989BA8911968C9162960FB6F894DEBF6A
S12353C00FBECDBFCF91DF911F910F91FF90EF90DF90CF90BF90AF909F908F907F906F908A
S12353E05F904F903F902F900895EF92FF920F931F93CF93DF93EC01FC01E258FF4F019073
S1235400F081E02D9881AFE3B0E08C9181FDFDCF1FBAF2BDE1BD90BD0FB6F894FA9AF99A7D
S12354200FBEFE01E258FF4F0190F081E02D2981AFE3B0E08C9181FDFDCF1FBACF01019692
S123544092BD81BD20BD0FB6F894FA9AF99A0FBEFE01E258FF4F0190F081E02D2C81AFE3C4
S1235460B0E08C9181FDFDCF1FBACF01049692BD81BD20BD0FB6F894FA9AF99A0FBEFE0140
S1235480E258FF4F0190F081E02D2D81AFE3B0E08C9181FDFDCF1FBACF0105960F2EF1E4E4
S12354A0EF2EFF24F02DF7019183808320BD0FB6F894FA9AF99A0FBE8E0102581F4FF8010A
S12354C060817181685F7F4FCE01C0960E940A27F80160817181645F7F4FCE0108960E94FC
S12354E00A27F80160817181605F7F4FCE010C960E940A27F801608171816C5E7F4FCE01A7
S123550040960E940A27F80160817181685E7F4FCE0144960E940A27F80160817181645E74
S12355207F4FCE0148960E940A27F80160817181605E7F4FCE018C589F4F0E940A27F80154
S1235540608171816C5D7F4FCE0180960E940A27F80160817181685D7F4FCE0184960E943B
S12355600A27F80160817181645D7F4FCE0188960E940A27F80160817181605D7F4FCE01B5
S12355808C960E940A27F801608171816C5C7F4FCE01C4960E940A27F80160817181685C24
S12355A07F4FCE01805C9F4F0E940A2712BCF7011082DF91CF911F910F91FF90EF9008958A
S12355C0CF92DF92EF92FF920F931F938C0182E80E941A2688E50E941A26F8018081880FD6
S12355E00E941A26F80181810E941A26F80182810E941A26F80183810E941A26F80184812D
S12356000E941A26F80185810E941A26F80186810E941A2680E00E941A260F2EFFEFCF2E77
S1235620FFE8DF2EF0E0EF2EF0E0FF2EF02DD701C6010197A109B109000001F0D1F7C895BA
S12356400000C801C0960E94DC26C80108960E94DC26C8010C960E94DC26D701C601019732
S1235660A109B109000001F0D1F7C8950000C80140960E94DC26C80144960E94DC26C80159
S123568048960E94DC26D701C6010197A109B109000001F0D1F7C8950000C8018C589F4F38
S12356A00E94DC26C80180960E94DC26C80184960E94DC26D701C6010197A109B10900009D
S12356C001F0D1F7C8950000C80188960E94DC26C8018C960E94DC26C801C4960E94DC26CF
S12356E0D701C6010197A109B109000001F0D1F7C8950000C801CC960E94DC26C801C896FF
S12357000E94DC26C801805C9F4F0E94DC26D701C6010197A109B109000001F0D1F7C895F9
S12357200000C8018C5B9F4F0E94DC26C801885B9F4F0E94DC26C801845B9F4F0E94DC26AB
S1235740D701C6010197A109B109000001F0D1F7C8950000C8018C599F4F0E94DC26C8018B
S12357608C5A9F4F0E94DC268DE70E941A261F910F91FF90EF90DF90CF900895DF93CF93BA
S123578000D000D0CDB7DEB7BC01CE01019644E050E02CEF36E20E94013C29813A814B8192
S12357A05C81622F732F842F952F0F900F900F900F90CF91DF9108952F923F924F925F9211
S12357C06F927F928F929F92AF92BF92CF92DF92EF92FF920F931F93DF93CF9300D000D023
S12357E0CDB7DEB79C838B8381E0AB81BC818C9314961C9280E090E0A0E4BFE3EB81FC813F
S123580084879587A687B7878DEC9CECACECBEE3EB81FC81808B918BA28BB38B20E030E02D
S123582040E050E0AB81BC8154962D933D934D935C935797EB81FC81208F318F428F538F69
S123584080E090E0A0E8BFE3EB81FC81848F958FA68FB78F80E090E0A0E8B0E4EB81FC81DA
S123586080A391A3A2A3B3A383E393E3A3E3BFE3EB81FC8184A395A3A6A3B7A380E090E073
S1235880A0EFB1E4EB81FC8180A791A7A2A7B3A780E090E0ACE8B2E4EB81FC8184A795A7AB
S12358A0A6A7B7A780E090E0A0E2B2E4EB81FC8180AB91ABA2ABB3AB80E090E0A0EAB0E468
S12358C0EB81FC8184AB95ABA6ABB7ABAB81BC81D8962D933D934D935C93DB97EB81FC8128
S12358E024AF35AF46AF57AFEB81FC81E05CFF4F80E090E0A0E8BEE380839183A283B38314
S1235900EB81FC8180899189A289B389EC58FF4F80839183A283B383EB81FC81E85BFF4F92
S12359202083318342835383EB81FC81E45AFF4F2083318342835383EB81FC81E258FF4F99
S12359400190F081E02DAFE3B0E08C9181FDFDCFCF01049692BD81BDF89A80B5AB81BC8184
S123596014968C93149714968C911497853030F014961C928B819C810E94F529EB81FC813E
S1235980E258FF4F0190F081E02DAFE3B0E08C9181FDFDCFF2BDE1BDF89A80B5EB81FC81E6
S12359A08083EB81FC81E258FF4F0190F081E02DAFE3B0E08C9181FDFDCFCF01019692BD21
S12359C081BDF89A80B5AB81BC8111968C931197FD01E258FF4F0190F081E02DAFE3B0E030
S12359E08C9181FDFDCFCF01029692BD81BDF89A80B5EB81FC818283EB81FC81E258FF4F21
S1235A000190F081E02DAFE3B0E08C9181FDFDCFCF01039692BD81BDF89A80B5AB81BC81C4
S1235A2013968C931397FD01E258FF4F0190F081E02DAFE3B0E08C9181FDFDCFCF01049668
S1235A4092BD81BDF89A80B5EB81FC818483EB81FC81E258FF4F0190F081E02DAFE3B0E05C
S1235A608C9181FDFDCFCF01059692BD81BDF89A80B5AB81BC8115968C93159781E08C939D
S1235A8014968C911497882321F081E014968C9303C0EB81FC811482AB81BC8114961C92A7
S1235AA01497FD01E258FF4F0190F081E02DAFE3B0E08C9181FDFDCFCF0106960F2EF1E49B
S1235AC0EF2EFF24F02DF70191838083F89A80B5AB81BC8116968C9316978D0102581F4F58
S1235AE0F8018081918108960E94BE2BAB81BC81D0966D937D938D939C93D397F8018081DB
S1235B0091810C960E94BE2BAB81BC8118966D937D938D939C931B97F80180819181409638
S1235B200E94BE2BAB81BC811C966D937D938D939C931F97EB81FC8184859585A685B78533
S1235B40E059FF4F80839183A283B383D8018D919C9144960E94BE2BEB81FC81608B718BEF
S1235B60828B938BD8018D919C9148960E94BE2BEB81FC81648B758B868B978BD8018D9167
S1235B809C914C960E94BE2BEB81FC81608F718F828F938FD8018D919C9180960E94BE2B97
S1235BA0EB81FC81EC58FF4F6083718382839383F8018081918184960E94BE2BAB81BC815A
S1235BC090966D937D938D939C939397F8018081918188960E94BE2BAB81BC8194966D93CA
S1235BE07D938D939C939797F801808191818C960E94BE2BAB81BC8198966D937D938D9394
S1235C009C939B97F80180819181C0960E94BE2BAB81BC819C966D937D938D939C939F9702
S1235C20F80180819181C4960E94BE2BAB81BC81D4966D937D938D939C93D797F8018081D5
S1235C409181C8960E94BE2BEB81FC81E05CFF4F608371838283938312BCD7011C926081AB
S1235C607181828193812FE632E143E85AE30E94C93C882364F4EB81FC81E05CFF4F8FE6F5
S1235C8092E1A3E8BAE380839183A283B383EB81FC81608971898289938920E030E040E0D0
S1235CA050E00E94C93C181654F080E090E0A0E2B1E4EB81FC81808B918BA28BB38BEB81C9
S1235CC0FC81EC58FF4F608171818281938120E030E040E050E00E94C93C181664F0EB81D2
S1235CE0FC81EC58FF4F80E090E0A0E2B1E480839183A283B383EB81FC81E05CFF4F6081E4
S1235D0071818281938120E030E040E050E00E94C93C181664F0EB81FC81E05CFF4F80E01A
S1235D2090E0A0E8BFE380839183A283B383AB81BC8190966D917D918D919C91939720E043
S1235D4030E040E050E00E94C93C181654F080E090E0A0E2B1E4EB81FC8180A391A3A2A35A
S1235D60B3A3AB81BC81D4966D917D918D919C91D79720E030E040E050E00E94C93C1816FC
S1235D8054F080E090E0A0E2B1E4EB81FC8184AB95ABA6ABB7ABAB81BC811C966D917D91A2
S1235DA08D919C911F97A05CBF4FBA83A9832D913D914D915C91EB81FC81E088F1880289BF
S1235DC013890E94613EA80197010E94CD3CEB81FC81E05AFF4F6083718382839383A98169
S1235DE0BA816D917D918D919C91EB81FC81EC58FF4F20813181428153810E94CD3CEB8191
S1235E00FC81EC59FF4F6083718382839383EB81FC81648575858685978520A131A142A113
S1235E2053A1E488F588068917892488358846885788A0A0B1A0C2A0D3A0A981BA816D9074
S1235E407D908D909C900E94613EA80197010E94613E7B018C01C601B501A40193010E94C4
S1235E60613E9B01AC01C201B1010E94653C9B01AC01C801B7010E94CD3CEB81FC81E859DF
S1235E80FF4F6083718382839383EB81FC81A488B588C688D788E488F5880689178960A1A6
S1235EA071A182A193A1A981BA812D913D914D915C910E94613E9B01AC01C801B7010E940C
S1235EC0653C9B01AC01C601B5010E94CD3CEB81FC81E459FF4F60837183828393830F90A7
S1235EE00F900F900F90CF91DF911F910F91FF90EF90DF90CF90BF90AF909F908F907F90DA
S1235F006F905F904F903F902F900895282F392FEFE3F0E0808181FDFDCF822F932F92BD17
S1235F2081BDF89A80B50895AF92BF92CF92DF92EF92FF920F931F93CF93DF938091A20268
S1235F409091A302A091A402B091A502A8958091DF05853809F494C08638C0F48B3579F1DC
S1235F608C3550F4843309F442C4853509F4EAC0833309F048C438C4813809F471C08338A4
S1235F8009F4D8C2803809F03EC4B8C2833909F447C4843950F48A3809F4F9C0813909F445
S1235FA09CC1883809F02FC416C1883909F4D5C1893909F421C4853909F025C468C28CE5CA
S1235FC00E941A2684E10E941A26C0E0D0E00F2EF3E1EF2EF4E0FF2EF02D0F2EFCECCF2ED6
S1235FE0FCE1DF2EF02DCE01880F991F880F991F8701080F191FF80180819181A281B381EF
S12360000E941A26F80180819181A281B381892F9A2FAB2FBB270E941A26F801808191810C
S1236020A281B381CD01AA27BB270E941A26F80180819181A281B3818B2F9927AA27BB2712
S12360400E941A26C6010197F1F7000000002196C530D10509F0C7CF83EA0E941A26E0C310
S123606082E08093DF058091220290E09695982F8827979587958D5E9C4F0E94E02AD0C320
S1236080A1EEB5E0FD0131912081922F80E07C01E30EF11C11978C91823009F43BC020E06C
S12360A030E00F2EFFEDCF2EF5E0DF2EF02DAFE3B0E001E410E060E470E04CEC5CE10F2E6A
S12360C0F0EEAF2EF5E0BF2EF02DA895F601E20FF31F3496E0818C9181FDFDCF1C92C901E1
S12360E08E0D9F1DE80199838883EB01E8830FB6F894FA9AF99A0FBECA010197F1F700004E
S123610000002F5F3F4FF501808190E0029728173907D8F286E80E941A2684E00E941A2680
S123612081E00E941A268E2D0E941A268F2D0E941A268091E00582500E941A2689E70E9421
S12361401A266EC3E1EEF5E091918081182F00E0090F111DC80166E87FE20E941D3CF82EFD
S1236160E92E85E50E941A2684E00E941A268F2D0E941A268E2D0E941A26802F0E941A26A6
S1236180812F0E941A268AEA0E941A2649C3E1EEF5E031912081922F80E0EC01C30FD11D32
S12361A08BE80E941A2683E00E941A26EFE3F0E0808181FDFDCFD2BDC1BDF89A80B50E94DE
S12361C01A268C2F0E941A268D2F0E941A2684E70E941A2625C389E80E941A2680E10E94B5
S12361E01A260F2EFFE3EF2EF2E0FF2EF02DE701888199810E941A2688819981892F0E9499
S12362001A26870104501040F801808191810E941A26E80188819981892F0E941A268701F2
S12362200C5F1F4FF801808191810E941A26E80188819981892F0E941A2687010E501040B7
S1236240F801808191810E941A26E80188819981892F0E941A2682E39BE20197F1F7000044
S1236260C89587010C501040F801808191810E941A26E80188819981892F0E941A2687016D
S12362800A501040F801808191810E941A26E80188819981892F0E941A268701085010408C
S12362A0F801808191810E941A26E80188819981892F0E941A26EAEFFFEFEE0EFF1EE7017E
S12362C0888199810E941A2688819981892F0E941A2686E70E941A26A3C282E90E941A26F7
S12362E080E10E941A268091220290E09695982F88279795879503E113E089599C4F0E9483
S1236300DC268091220290E09695982F882797958795C896800F911F0E94DC268091220273
S123632090E09695982F8827979587950896800F911F0E94DC268091220290E09695982FE8
S1236340882797958795885B9F4F800F911F0E94DC268DE60E941A2663C287E90E941A26C2
S123636081E10E941A260F2EF3E3EF2EF2E0FF2EF02DF701808191810E941A268701E7012C
S123638089919991892F0E941A26888199810E941A2688819981892F0E941A260C5F1F4F80
S12363A0F801808191810E941A26E80188819981892F0E941A268091A2029091A302A09199
S12363C0A402B091A5020E941A2660914B0370914C0380914D0390914E0320E030E040E2B5
S12363E051E40E94613E0E943A3DDC01CB010E941A268701025F1F4FF801808191810E947A
S12364001A26E80188819981892F0E941A2687B52AE0829FC0011124C29769E170E00E94A0
S1236420363F862F0E941A2686E69EE00197F1F70000F7017096808191816AE070E00E9495
S1236440223F862F0E941A26ECE0F0E0EE0EFF1EE701888199810E941A2688819981892FC3
S12364600E941A2680911E0590911F050E941A2680911E0590911F05892F0E941A268091B7
S12364808F020E941A2688E60E941A26C9C186E90E941A2680E10E941A268091220290E072
S12364A09695982F88279795879503E113E089599C4F0E94DC2685E892E00E94DC26809113
S12364C0220290E09695982F8827979587950896800F911F0E94DC268091220290E09695EA
S12364E0982F882797958795885B9F4F800F911F0E94DC2689E60E941A2692C18091E1058B
S12365008093220280912202882331F080912202813011F01092220280E80E941A2681E0E7
S12365200E941A26809122020E941A268FE70E941A2676C184E80E941A2684E20E941A2639
S123654080910D0190910E010E941A2680910D0190910E01892F0E941A2680910F010E945A
S12365601A26809110010E941A260FEF17E4C8010197F1F7000000C080911101909112017A
S12365800E941A268091110190911201892F0E941A2680913301909134016AE070E00E944D
S12365A0223F862F0E941A2680913301909134016AE070E00E94223F872F0E941A268091FE
S12365C01301909114016AE070E00E94223F862F0E941A2680911301909114016AE070E044
S12365E00E94223F872F0E941A2680911501909116016AE070E00E94223F862F0E941A2669
S1236600C8010197F1F7000000C080911501909116016AE070E00E94223F872F0E941A26D9
S123662080911701909118016AE070E00E94223F862F0E941A2680911701909118016AE012
S123664070E00E94223F872F0E941A2680911B0190911C016AE070E00E94223F862F0E94EC
S12366601A2680911B0190911C016AE070E00E94223F872F0E941A26809157019091580153
S12366800E941A268091570190915801892F0E941A26C8010197F1F7000000C080911D015F
S12366A090911E016AE070E00E94223F862F0E941A2680911D0190911E016AE070E00E94B7
S12366C0223F872F0E941A2680913501909136016AE070E00E94223F862F0E941A268091D9
S12366E03501909136016AE070E00E94223F872F0E941A2680911F01909120010E941A267E
S123670080911F0190912001892F0E941A26C8010197F1F7000000C0809123010E941A2648
S1236720809124010E941A2680912501909126016AE070E00E94223F862F0E941A26809179
S12367402701909128016AE070E00E94223F862F0E941A2680912B010E941A2680912C0132
S12367600E941A26C8010197F1F7000000C080912D0190912E016AE070E00E94223F862F49
S12367800E941A2680912D0190912E016AE070E00E94223F872F0E941A2680912F019091ED
S12367A030016AE070E00E94223F862F0E941A2680912F01909130016AE070E00E94223F40
S12367C0872F0E941A2680913101909132010E941A268091310190913201892F0E941A2673
S12367E08BE70E941A261CC00E94830219C00E9482070E946D0A14C0F894E091ED01F091E1
S1236800EE0109950DC08EE80E941A2681E00E941A268091DF050E941A2681E70E941A265E
S1236820EFEDF5E011928081882391F020E030E04FED55E0DA011196FA01E20FF31F32960A
S123684010822F5F3F4F8C9190E028173907A0F31092E005DF91CF911F910F91FF90EF9032
S1236860DF90CF90BF90AF900895AF92BF92CF92DF92EF92FF920F931F93CF93DF93382F16
S1236880492FC62E2DE088E190E00FB6F894A895809360000FBE20936000662309F4C0C0BB
S12368A0D32E232F342FE9010F2EF0EEEF2EF5E0FF2EF02D0FED15E0AA246894A1F8BB24AA
S12368C0B39480910303882309F05FC08881F80180838081833309F447C08081843309F41E
S12368E043C08081853509F43FC080818835E1F180818B35C9F180818136B1F180818536B9
S123690099F180818F3681F18081803769F18081873751F18081893739F18081803821F1E8
S123692080818A3709F180818138F1F080818338D9F080818438C1F080818538A9F08081B1
S1236940883891F080818A3879F08081813961F08081833949F08081853931F08081883922
S123696019F08081893919F4B092030353C08FE80E941A268B2D0E941A26F80180810E9450
S12369801A2680E70E941A2645C080910303813059F48881F70180838081833310F01092F3
S12369A00303A092030336C020910303F701808130E090E002962817390791F4F8018081D9
S12369C0809580930303909103038881891729F4109203030E94942F1DC0109203031AC02C
S12369E0809103038230B0F020910303F701808130E090E002962817390764F48091030374
S1236A009881F801E80FF11D9083809103038F5F8093030321969E012D192C1508F451CF31
S1236A20DF91CF911F910F91FF90EF90DF90CF90BF90AF900895000000000000000000002B
S1236A400000000000000000000000000000000000000000000090E0209117063091180615
S1236A60280F391F22953295307F3227207F3227282B392B2F703F70E8E2F0E08081806184
S1236A80808380818F7B808348E0AFE5B0E080818F7E808380818F7D80839C91917092951F
S1236AA0990F907E80818F7D892B8083000000000000000000000000000000000000000058
S1236AC000000000000000000000000080818061808341500000000000000000000000003C
S1236AE00000000000000000000000000000000000000000442389F00000000000000000B2
S1236B00000000000000000000000000000000000000000000000000BACF40E1E8E2F0E02D
S1236B20AFE5B0E080818F7E808380818F7D8083369527959C9191709295990F907E808179
S1236B408F7D892B80838081806180834150000000000000000000000000000000000000F8
S1236B60000000000000000000000000000000000000000000000000000000000000000011
S1236B800000000000000000000000000000000000000000000000000000000000000000F1
S1236BA00000000000000000000000000000442309F0B8CF3093180620931706E8E2F0E09F
S1236BC08081806480838081806180836A3F39F480E791E00197F1F70000000008958CECA1
S1236BE09CE10197F1F700000000089580910703E4E1F2E0E80FF11D808190910603890F7D
S1236C0068EF0E941B35089580930603609307030E94F635089510920603809107038F5F53
S1236C2080930703823010F0109207030E94F63508958A3029F40E940B360E94F635089547
S1236C406AEF0E941B35809106038F5F809306030895CF93DF93FC01009751F080818823CF
S1236C6039F0EF010E941936219688818823D1F7DF91CF9108956AEF0E941B35089588E313
S1236C8068EF0E941B3508958BE368EF0E941B35089581E068EF0E941B35109206031092BF
S1236CA0070308950F931F93E7E2F0E08081806480838081806180838081806280831092E7
S1236CC01406E8E2F0E08081806480838081806180838FEF97EDA0E0B0E00197A109B10921
S1236CE0000001F0D1F7C895000081E068EF0E941B350CEC1CE1C8010197F1F70000000092
S1236D0088E368EF0E941B358FE068EF0E941B3586E068EF0E941B3581E068EF0E941B35AA
S1236D20C8010197F1F7000000001F910F9108950E9452360E940B368FEE91E00E9429361D
S1236D4008958F929F92AF92BF92CF92DF92EF92FF920F931F93DF93CF93CDB7DEB72997C9
S1236D600FB6F894DEBF0FBECDBF8C01F62EE42EDE011196EBE0F2E089E001900D92815078
S1236D80E1F749E00F2EF9E0AF2EBB24F02D6E010894C11CD11C0F2EFEE28F2EF02D992476
S1236DA0FF2071F09501241B31098F2D90E02817390730F04150F601E40FF11D8082F92CC5
S1236DC04150F601E40FF11DC8016AE070E00E94223F805D8083C8016AE070E00E94223F7A
S1236DE0862F972F8C010115110511F4FF2019F085E08F15A8F689E0182F1E19193068F4FB
S1236E007E010894E11CF11CF701E10FF11D80810E9419361F5F1930B8F329960FB6F894DF
S1236E20DEBF0FBECDBFCF91DF911F910F91FF90EF90DF90CF90BF90AF909F908F900895E3
S1236E408F929F92AF92BF92CF92DF92EF92FF920F931F93DF93CF93CDB7DEB72A970FB69F
S1236E60F894DEBF0FBECDBF8C01F62E842EDE011196E2E0F2E089E001900D928150E1F7CD
S1236E80112314F01A8607C0109501951F4F8DE2898381E08A8749E00F2EF9E0AF2EBB24BE
S1236EA0F02D6E010894C11CD11C0F2EFEE29F2EF02DEE24FF2071F09501241B31098F2D78
S1236EC090E02817390730F04150F601E40FF11D9082FE2C4150F601E40FF11DC8016AE03E
S1236EE070E00E94363F805D8083C8016AE070E00E94363F862F972F8C010115110511F494
S1236F00FF2019F085E08F15A8F68A858130A1F498E0BE016F5F7F4F292F30E0FB01E20F21
S1236F20F31F8081803231F4FE01E20FF31F8DE2818302C09150F0CF89E0182F1819193062
S1236F4068F47E010894E11CF11CF701E10FF11D80810E9419361F5F1930B8F32A960FB6CD
S1236F60F894DEBF0FBECDBFCF91DF911F910F91FF90EF90DF90CF90BF90AF909F908F90B3
S1236F800895EFE3F0E0808181FDFDCF84E893E092BD81BDF89A80B580931203EFE3F0E066
S1236FA0808181FDFDCF85E893E092BD81BDF89A80B580932505EFE3F0E0808181FDFDCF24
S1236FC086E893E092BD81BDF89A80B580933F05EFE3F0E0808181FDFDCF87E893E092BD03
S1236FE081BDF89A80B580932D04089580911203882359F480912505813039F480913F051B
S123700090E0823019F491E001C090E0892F089580912D04811181E00895AF92BF92CF9281
S1237020DF92EF92FF920F931F93CF93DF93982F7A018B01E90180910803891721F010927A
S12370401D0690930803943109F447C0953140F4992381F0892F8950823008F0DDC017C03C
S1237060903209F47CC0983209F495C09E3109F0D3C054C082E390E09B8B8A8B81E090E0A5
S12370809987888784EF91E09D8B8C8BC5C0CC24DD246894C3F8CC0EDD1EC801B7012CEB00
S12370A032E040E050E00E94493FF60131832083215233402CF080E293E0F601918380830D
S12370C080911D0624E333E0281B31093D8B2C8B82E390E09B8B8A8B9FC0FE0138968EE5B3
S12370E091E09183808380911D0690E0880F991F82549F4F9183808320911D0684E393E088
S1237100821B91099D8B8C8B80911D066FE00E94163F90E0C2969B8B8A8B7EC0FE0138966D
S12371208EE591E09183808380911D0690E0880F991F82549F4F9183808320911D0684E347
S123714093E0821B91099D8B8C8B80911D0664E10E94163F90E0CC969B8B8A8B5DC0FE01A9
S123716038968EE591E09183808380911D0690E0880F991F82549F4F9183808320911D06A0
S123718084E393E0821B91099D8B8C8B82E390E09B8B8A8B41C0FE01389682E593E09183CF
S12371A0808380911D0690E0880F991F909581959F4F8E5A9C4F9183808380911D0690E01E
S12371C088539F4F9D8B8C8B0F2EF2E1AF2EBB24F02DAC0EBD1EF501C080D180F3E3CF16E3
S12371E0D104D4F0C801B70124EF31E040E050E00E94493F8091190690911A06A0911B0610
S1237200B0911C06281739074A075B0769F1C6010197F50191838083C801B70124EF31E06A
S123722040E050E00E94493F822F932FA42FB52F9C01AD018091190690911A06A0911B0698
S1237240B0911C06281739074A075B0769F080911D068F5F80931D062093190630931A062F
S123726040931B0650931C068A899B899C01220F331F880F991F880F991F880F991F280F96
S1237280391F3F8B2E8BDF91CF911F910F91FF90EF90DF90CF90BF90AF900895282F392F29
S12372A0EFE3F0E0808181FDFDCF822F932F92BD81BDF89A80B50895282F392FEFE3F0E018
S12372C0808181FDFDCF1FBA822F932F92BD81BD60BD0FB6F894FA9AF99A0FBE0895CF9226
S12372E0DF92EF92FF920F931F93CF93DF93C0E0D0E004EA16E00F2EFEE2CF2EF4E0DF2EB0
S1237300F02D0F2EFCE5EF2EF9E3FF2EF02DA895CE01880F991FF601E80FF91F60817181B7
S1237320C801A7010E944F3C21960E5F1F4FC837D10569F76091200570912105809122056F
S12373409091230520E030E040E251E40E94613E0E943A3D9B01AC0180EA96E0B9014CE50B
S123736059E30E944F3CDF91CF911F910F91FF90EF90DF90CF900895EF92FF920F931F93A1
S1237380CF93DF93EB018D3C910540F4EEE2F4E08081918101969183808314C0885C9040A9
S12373A065E070E00E94223F683708F067E7E62FF0E0EE0FFF1FE25DFB4F80819181019619
S12373C0918380836091200570912105809122059091230520E030E04EEB52E40E94613E14
S12373E07B018C01BE01660F771F660F771F6C0F7D1F80E090E00E94663D9B01AC01C8016D
S1237400B7010E94653C20E030E048EC52E40E94CD3C6093200570932105809322059093AA
S12374202305809111038F5F80931103893720F00E946F3910921103DF91CF911F910F91F6
S1237440FF90EF900895AF92BF92CF92DF92EF92FF920F931F93CF93DF93C0E0D0E004EAA1
S123746016E00F2EFEE4AF2EF9E3BF2EF02D0F2EFEE2CF2EF4E0DF2EF02DA895C801B5015C
S12374800E941D3C9E01220F331FF601E20FF31F91838083808191818D5D9F4F40F0CE01D0
S12374A0880F991FF601E80FF91F1182108221960E5F1F4FC837D10501F780EA96E06EE4BD
S12374C079E30E941D3C6AE070E00E94223F80E090E00E94663D609320057093210580934B
S12374E02205909323056091200570912105809122059091230520E030E849E854E40E9435
S1237500183E181664F480E090E8AEE5B4E48093200590932105A0932205B0932305DF91D2
S1237520CF911F910F91FF90EF90DF90CF90BF90AF900895EF92FF920F931F93CF93DF9356
S1237540C4E4D6E00F2EF3E1EF2EF4E0FF2EF02D0EE419E3CE01845496408E0D9F1DBE01FC
S123756044E050E098010E94013C249686E0C835D80781F712BC11BCDF91CF911F910F910C
S1237580FF90EF900895EF92FF920F931F9303E114E00F2EFCE5EF2EF9E3FF2EF02D84E435
S12375A096E0B80144E050E097010E94333CB8016C5F7F4F88E496E044E050E097010E94D9
S12375C0333CB801685F7F4F8CE496E044E050E097010E94333CB801645F7F4F80E596E0E2
S12375E044E050E097010E94333C005F1F4F84E596E0B80144E050E097010E94333C1F9178
S12376000F91FF90EF900895EF92FF920F931F936091A9017091AA018091AB019091AC01E3
S123762020E63AEE40E050E00E94493F790100E010E08091090390910A03A0910B03B09189
S12376400C03E816F9060A071B0709F4C2C0E3E1F4E080819181A281B381209109033091E8
S12376600A0340910B0350910C03821B930BA40BB50B8E0D9F1DA01FB11F80839183A2835E
S1237680B38380918F02853148F4833170F5893089F08A3051F1882369F077C0803251F0A7
S12376A0813220F48E3108F470C03AC0883209F06CC051C0E7E1F4E080819181A281B38124
S12376C02091090330910A0340910B0350910C03821B930BA40BB50B8E0D9F1DA01FB11FBC
S12376E080839183A283B38350C0EBE1F4E080819181A281B3812091090330910A0340919E
S12377000B0350910C03821B930BA40BB50B8E0D9F1DA01FB11F80839183A283B38335C070
S1237720EFE1F4E080819181A281B3812091090330910A0340910B0350910C03821B930BA2
S1237740A40BB50B8E0D9F1DA01FB11F80839183A283B3831AC0E3E2F4E080819181A281B5
S1237760B3812091090330910A0340910B0350910C03821B930BA40BB50B8E0D9F1DA01FB7
S1237780B11F80839183A283B38380910D0390910E03A0910F03B09110034496A11DB11D53
S12377A08E159F05A007B10750F40E94C33AE0920D03F0920E0300930F031093100312BCFE
S12377C011BCE0920903F0920A0300930B0310930C031F910F91FF90EF9008950E94C33ADE
S12377E01092090310920A0310920B0310920C0310920D0310920E0310920F0310921003F9
S12378000895A0E0B0E0E7E0FCE30C94753F7C01EB018A01690109C0CE012196F60109957B
S1237820F70181937F010150104001151105A1F7CDB7DEB7E8E00C94913FDF92EF92FF927F
S12378400F931F937B018C01FB010995D82EC8010196F7010995982F8D2D1F910F91FF90D1
S1237860EF90DF900895A0E0B0E0E9E3FCE30C94753FEC017B018A01690109C0CE012196BD
S1237880F70161917F01F60109950150104001151105A1F7CDB7DEB7E8E00C94913FDF92BE
S12378A0EF92FF920F931F93D72E7A018C01FA010995C80101966D2DF70109951F910F91D8
S12378C0FF90EF90DF9008955058BB27AA270ED075C166D130F06BD120F031F49F3F11F470
S12378E01EF45BC10EF4E095E7FB51C1E92F77D180F3BA17620773078407950718F071F4D0
S12379009EF58FC10EF4E0950B2EBA2FA02D0B01B90190010C01CA01A0011124FF27591B7B
S123792099F0593F50F4503E68F11A16F040A22F232F342F4427585FF3CF469537952795CA
S1237940A795F0405395C9F77EF41F16BA0B620B730B840BBAF09150A1F0FF0FBB1F661FA0
S1237960771F881FC2F70EC0BA0F621F731F841F48F4879577956795B795F7959E3F08F0B3
S1237980B3CF9395880F08F09927EE0F979587950895D9D008F481E008950CD00FC107D1E1
S12379A040F0FED030F021F45F3F19F0F0C0511139C1F3C014D198F39923C9F35523B1F326
S12379C0951B550BBB27AA2762177307840738F09F5F5F4F220F331F441FAA1FA9F333D040
S12379E00E2E3AF0E0E830D091505040E695001CCAF729D0FE2F27D0660F771F881FBB1FE3
S1237A00261737074807AB07B0E809F0BB0B802DBF01FF2793585F4F2AF09E3F510568F0BE
S1237A20B6C000C15F3FECF3983EDCF3869577956795B795F7959F5FC9F7880F911D9695C0
S1237A40879597F90895E1E0660F771F881FBB1F621773078407BA0720F0621B730B840BB3
S1237A60BA0BEE1F88F7E095089504D06894B111D9C00895BCD088F09F5790F0B92F9927B5
S1237A80B751A0F0D1F0660F771F881F991F1AF0BA95C9F712C0B13081F0C3D0B1E0089521
S1237AA0C0C0672F782F8827B85F39F0B93FCCF3869577956795B395D9F73EF490958095B8
S1237AC0709561957F4F8F4F9F4F0895E89409C097FB3EF490958095709561957F4F8F4F86
S1237AE09F4F9923A9F0F92F96E9BB279395F695879577956795B795F111F8CFFAF4BB0F12
S1237B0011F460FF1BC06F5F7F4F8F4F9F4F16C0882311F096E911C0772321F09EE8872F01
S1237B20762F05C0662371F096E8862F70E060E02AF09A95660F771F881FDAF7880F96959C
S1237B40879597F90895990F0008550FAA0BE0E8FEEF16161706E807F907C0F01216130631
S1237B60E407F50798F0621B730B840B950B39F40A2661F0232B242B252B21F408950A26EB
S1237B8009F4A140A6958FEF811D811D089597F99F6780E870E060E008959FEF80EC0895AF
S1237BA000240A941616170618060906089500240A9412161306140605060895092E039459
S1237BC0000C11F4882352F0BB0F40F4BF2B11F460FF04C06F5F7F4F8F4F9F4F089557FD3A
S1237BE09058440F551F59F05F3F71F04795880F97FB991F61F09F3F79F087950895121654
S1237C0013061406551FF2CF4695F1DF08C0161617061806991FF1CF869571056105089413
S1237C200895E894BB2766277727CB0197F908958ADF08F48FEF08950EF0A6C0AECF6894C4
S1237C40A6CFD5DFC8F39923D1F3C6F3DF93CF931F930F93FF92C92FDD2788232AF02197D1
S1237C60660F771F881FDAF720E030E040E85FEB9FE3883920F0803E30F021968F7725DE0A
S1237C80E0E7F0E003C021DEEDE9F0E08BD08B01BE01EC01FB2E6F5771097595771F880BB2
S1237CA0990B16DF28E132E741E35FE316D0AF2D9801AE01FF900F911F91CF91DF9116DEF2
S1237CC07DCF0BD07BCF6CDF28F071DF18F0952309F05DCF62CF1124A5CF81DFA0F3959F96
S1237CE0D1F3950F50E0551F629FF001729FBB27F00DB11D639FAA27F00DB11DAA1F649F5A
S1237D006627B00DA11D661F829F2227B00DA11D621F739FB00DA11D621F839FA00D611D11
S1237D20221F749F3327A00D611D231F849F600D211D822F762F6A2F11249F5750408AF032
S1237D40E1F088234AF0EE0FFF1FBB1F661F771F881F91505040A9F79E3F510570F017CF28
S1237D6061CF5F3FECF3983EDCF3869577956795B795F795E7959F5FC1F7FE2B880F911D12
S1237D809695879597F908959F3F31F0915020F4879577956795B795880F911D969587957B
S1237DA097F90895DF93CF931F930F93FF92EF92DF927B018C01689405C0DA2EEF018DDFB9
S1237DC0FE01E894A5912591359145915591AEF3EF018CDDFE019701A801DA9479F7DF902F
S1237DE0EF90FF900F911F91CF91DF910895629FD001739FF001829FE00DF11D649FE00DD3
S1237E00F11D929FF00D839FF00D749FF00D659FF00D9927729FB00DE11DF91F639FB00D8F
S1237E20E11DF91FBD01CF0111240895991B79E004C0991F961708F0961B881F7A95C9F773
S1237E4080950895AA1BBB1B51E107C0AA1FBB1FA617B70710F0A61BB70B881F991F5A95E9
S1237E60A9F780959095BC01CD01089597FB092E07260AD077FD04D0E5DF06D000201AF41C
S1237E80709561957F4F0895F6F7909581959F4F0895A1E21A2EAA1BBB1BFD010DC0AA1FCB
S1237EA0BB1FEE1FFF1FA217B307E407F50720F0A21BB30BE40BF50B661F771F881F991F6B
S1237EC01A9469F760957095809590959B01AC01BD01CF0108952F923F924F925F926F9283
S1237EE07F928F929F92AF92BF92CF92DF92EF92FF920F931F93CF93DF93CDB7DEB7CA1B7F
S1237F00DB0B0FB6F894DEBF0FBECDBF09942A88398848885F846E847D848C849B84AA841D
S1237F20B984C884DF80EE80FD800C811B81AA81B981CE0FD11D0FB6F894DEBF0FBECDBFCA
S1237F40ED010895F894FFCF2043616C6962726174696E6700E8050164FA007E042C012895
S1237F60002C015E019001C8003200502858021E006400190A64002C0190011E00B00496E5
S1237F80000520038A02F4010801C800140A0601015802140A0A0A179F023D00C01C41F4AB
S1237FA0012828E203D703C903B603A003840363033C030F03DE02A902720239020002C942
S1237FC0019501640138010F01EC00CC00B100990084007200630056004B004100390032B0
S1237FE0002B00260022001E001A0017001500120064000000640000002500250025002538
S12380000025002800280028002800280001020408100810204080E2041B5B481B5B324AC2
S1238020000D0A002020202020202020206F12833A0000803F00E04D5254656368004C6158
S12380406D6264610054657374002020202020202020202020202020202020200040145400
S5030403F5
